S01A000066726565646F6D5F626F6F746C6F616465722E737265639E
S1130000F0C6FF1F11040000EB040000AD45000022
S113001000000000000000000000000000000000DC
S1130020000000000000000000000000EB040000DD
S11300300000000000000000EB040000EB040000DE
S1130040817A0000897A0000917A0000997A000090
S1130050A17A0000A97A0000D97A0000D97A0000B8
S1130060D97A0000D97A00006D480000D97A0000DE
S1130070116A0000176A000043670000B17A0000AB
S1130080D97A0000D97A00001B0E0000D97A00004A
S1130090D97A0000D97A0000D97A0000D97A000010
S11300A0398F0000D97A0000D97A0000D97A00008B
S11300B02D460000334600003F4600004546000040
S11300C0D97A0000D97A0000D97A0000D97A0000E0
S11300D077480000316A0000D97A00004D670000BB
S11300E0D97A0000D97A0000D97A0000D97A0000C0
S11300F0D97A0000D97A0000D97A0000D97A0000B0
S1130100D97A0000D97A0000D97A0000D97A00009F
S1130110D97A0000D97A0000D97A0000D97A00008F
S1130120B97A0000C17A0000C97A0000D17A0000CF
S1130130D97A0000D97A0000D97A0000D97A00006F
S1130140FFFFFFFFFFFFFFFFFFFFFFFFFFFFFFFFBB
S1130150FFFFFFFFFFFFFFFFFFFFFFFFFFFFFFFFAB
S1130160FFFFFFFFFFFFFFFFFFFFFFFFFFFFFFFF9B
S1130400FFFFFFFFFFFFFFFFFFFFFFFFFE3DFFFFBB
S113041072B60E480E49886000220023002400258D
S113042000260027B846B946BA46BB46BC4609482A
S1130430854609488047094880470948804762B68D
S113044000200021074A9047FEE70000000000005A
S113045000ED00E0F0C6FF1FE17A0000BD3F0000A0
S11304600140000077380000000000000000000098
S1130470002A01D101207047F0B41F46034603242B
S11304802340002B09D00424E31A0170013008240E
S1130490E141521E26D05B1EF7D1042A1ADB13D089
S11304A0002F11D00C460D460E46102A02DB72C0F6
S11304B0103AFAE70C2A02DB32C00C3AFAE7082AAF
S11304C002DB12C0083AFAE7042A03DB01600430B5
S11304D0121FF9E7002A05D0017001300824E14118
S11304E0521EF7D1F0BC00207047FEE769230000DC
S11304F000000000912300000000000073240000AD
S1130500C125000053240000E924000099260000BE
S1130510000000004727000000000000C72300007F
S113052000000000A3230000E9240000B12600001D
S11305300000000021270000000000002B23000021
S113054000000000F523000000000000000000008F
S1130550000000005B270000000000008727000067
S113056000000000BD270000C12500000924000090
S1130570000000000000000000000000000102462E
S1130580BD38000081390000000000009D390000E2
S1130590393A0000193C0000493C0000A13C00002D
S11305A0B13C0000453D0000853E00000000000015
S11305B0C33A0000D53B0000113B0000293900007C
S11305C0E53D000000000000000000000000000005
S11305D000000000154400002944000045440000C8
S11305E00000000099930000A3930000AD93000065
S11305F000000000000000001947000065470000EB
S1130600BD4700000000000000000000F1470000AA
S11306100100000051130000000000000000000071
S113062085290000B5290000F9290000E92A000005
S113063000000000252B000057670000A1670000A0
S113064055680000000000000000000091680000F0
S113065029690000AF690000C969000000000000BA
S113066000000000FD69000075430000DD4100004A
S11306700942000099420000D542000055420000A2
S113068052656164790D0A005472616E7366657215
S113069072696E670D0A0000537563636573730DA9
S11306A00A0000004661696C7572650D0A0000005D
S11306B0EB3C904D5357494E342E3100020101005A
S11306C0022000FF7FF08000010001000100000013
S11306D0FF7F0000000029313233344B696E6574AA
S11306E06973205553420000F0FFFFFFFFFFFFFF37
S11306F0FFFFFFFFFFFF000046534C204C6F616477
S11307006572200800000000000000000000006086
S11307102C42000000000000412E006600730065BA
S11307200076000F00DA65006E0074007300640048
S113073000000000FFFFFFFF46534556454E7E3143
S113074020202012000000602C422C420000006097
S11307502C4202000000000042650072005F006944
S1130760006E000F00A86400650078000000FFFF21
S1130770FFFF0000FFFFFFFF012E006D0065007406
S11307800061000F00A864006100740061005F0054
S11307906E000000650076004D45544144417E31B1
S11307A020202022000000602C422C420000006027
S11307B02C42000000000000412E00540072006131
S11307C00073000F00256800650073000000FFFF40
S11307D0FFFF0000FFFFFFFF5452415348457E31A5
S11307E020202022000000602C422C4200000060E7
S11307F02C4200000000000042200049006E006608
S1130800006F000F007272006D00610074006900D7
S11308106F0000006E000000015300790073007443
S11308200065000F00726D00200056006F006C0020
S1130830750000006D00650053595354454D7E31D9
S113084020202016000000602C422C420000006092
S11308502C42030000000000494E464F2020202077
S113086054585420000000602C422C4200000060C8
S11308702C420500010000005354415455532020DC
S113088054585420000000602C422C4200000060A8
S11308902C420600010000002E20202020202020D1
S11308A020202032000000602C422C420000006016
S11308B02C420200000000002E2E202020202020A8
S11308C020202010000000602C422C420000006018
S11308D02C420000000000004E4F5F4C4F47202088
S11308E020202020080000602C422C4200000060E0
S11308F02C420000000000007B003300370032006F
S1130900300033004200460038002D004600440009
S1130910380033002D0034003300320031002D0044
S113092041003400430034002D00390041003900F7
S113093041004200460038004600420043004600A1
S113094044007D00000000002E20202020202020D4
S113095020202032000000602C422C420000006065
S11309602C420300000000002E2E202020202020F6
S113097020202010000000602C422C420000006067
S11309802C4200000000000042470075006900642A
S11309900000000F00FFFFFFFFFFFFFFFFFFFFFF4F
S11309A0FFFF0000000000000149006E00640065C4
S11309B00078000F00FF6500720056006F006C00A5
S11309C0750000006D006500494E444558457E3170
S11309D020202020000000602C422C4200000060F7
S11309E02C4204004D00000049400000514000002A
S11309F05D4000006D4000000000000000000000A9
S1130A0001000000000000005D0D00005006000021
S1130A1060060000A40A00000200000001000000BB
S1130A209F0D00003806000048060000A40A0000DC
S1130A300400000001000000D10D0000F8050000D2
S1130A4008060000A40A00001000000000000000D6
S1130A5000000000C00A000000000000D00A0000EE
S1130A600000000000000000000000000000000082
S1130A70000000000000000075730000AF73000068
S1130A80D5740000AF75000058AAFF1F492F00005D
S1130A90472D0000532F0000632F0000432E000059
S1130AA0732F0000C9760000D5760000457700005A
S1130AB0FB770000CD76000007780000A9760000DF
S1130AC0298B0000498C0000538D0000958D000097
S1130AD0C98D0000F58D0000858E0000218F000077
S1130AE0318F0000358F00000000000038B505008C
S1130AF0434C002323620020002103C4083C22004D
S1130B00083203C22200103203C263623D4800F07F
S1130B10B0F8183403C43C49280000F090F931BD02
S1130B2080B500F0A0F901BD70B50C00344D296A00
S1130B3007291CD1696A884219D100F0CFF896269A
S1130B40F60001010A1A03CD030003CD19181000A1
S1130B5000F0B8F90A214843310000F0B3F9401D10
S1130B600A2100F0AFF970432060002070BD01201D
S1130B7070BDF1B582B000F076F804000D00204E8F
S1130B80376A7F1C3000183003C800900191300090
S1130B90103003C82B00221A8B4100980199994206
S1130BA003D801D3904200D201273762012F06D027
S1130BB0042F09D0052F0FD0072F11D01CE030C609
S1130BC0083E0298706217E00CCE083E2900A01A75
S1130BD0994103C6083E0FE03000083030C00BE0F6
S1130BE0300008300CC82900A01A9941320008329C
S1130BF003C2029800F037F9103630C6F7BD000082
S1130C0020A9FF1F80380100730B000010B52D4888
S1130C100168802212040A43026000202A49086005
S1130C202A490022D2430A6188610124CC6188697F
S1130C30042303438B618869204388610A60CC6084
S1130C408C6000F009FAC000214900F03BF900284B
S1130C5000D101201F49086010BD1B480168022211
S1130C600A43026070471C4801684068C043C94396
S1130C70704700B50021174A1268002300F02EFACD
S1130C80C0084A071043C90800BDD0B50400FFF7E7
S1130C90EAFF06000F00200000210E4A126800231C
S1130CA000F01CFAC0084A071043C90836184F411F
S1130CB0FFF7D9FFB942FBD301D8B042F8D3D0BD76
S1130CC0000000003C8004400070034000710340B9
S1130CD040420F004CAAFF1FE070034080B500F0B3
S1130CE0BBF902BD10B58207D30EFF249C40E2433A
S1130CF08907090E9940030004D566481B071B0F9A
S1130D00083B00E064489B089B00C01803681A4035
S1130D101143016010BD8900401801685F4B0B400E
S1130D201104F02212030A401A430260704789003A
S1130D304158C801C00F704709E01202E023DB00EC
S1130D40134020221A4389004250704700BF120208
S1130D50E023DB001340890043507047002800D093
S1130D60704710B54E4C002903D002290CD003D390
S1130D7010BD2064606410BDA00D20644948016862
S1130D80494A0A40026010BD032210212000FFF7E7
S1130D90D3FF032211212000FFF7CEFF10BD01284D
S1130DA000D0704710B5414C002902D0022904D06C
S1130DB010BD0020A062E06210BD02220B212000C1
S1130DC0FFF7BBFF02220A212000FFF7B6FF10BD88
S1130DD0012800D0704710B5354C002902D00229F3
S1130DE006D010BD002020616061A061E06110BDEB
S1130DF0072204212000FFF7A9FF07220521200074
S1130E00FFF7A4FF072206212000FFF79FFF072218
S1130E1007212000FFF79AFF10BD80B5102120485C
S1130E20FFF785FF002809D022480168080005D093
S1130E30002088470020C0431F49086001BD10B549
S1130E400C0000280ED101211220FFF74BFF802057
S1130E50C0021A4908600A2210211148FFF75BFFFB
S1130E601448046010BD002800D0704780B580206D
S1130E70C0021349086000211220FFF733FF00224B
S1130E8010210748FFF747FF00200A49086001BD09
S1130E90000000001CED00E000E400E0FFFFF0FFB4
S1130EA000A0044054F00F40FFFFFEFF00B00440D8
S1130EB000C0044054AAFF1FA0A0044000E100E0C9
S1130EC080E100E0094214D088420FD30122030CD0
S1130ED001D100041204002300185B418B4200D3AB
S1130EE05B1A5241F8D3190010007047010000202A
S1130EF0704708B500F00CF908BD0268531C036084
S1130F001170704700206649820089180A68654B91
S1130F1013400B60401C0E28F5D304207047F1B534
S1130F2001260023002434305D49A022D200009F12
S1130F30002F01D101240CE08769042F43D20768F4
S1130F40002F00D100268768002F00D00123002E37
S1130F5028D04A608A600A614A61002C36D1E024B4
S1130F60E4004568002D00D0CC618569022D01D0D4
S1130F70032D01D10A60CA608569032D0ED10A626E
S1130F808A624A628A61009DCE267600AD192E6877
S1130F90002E02D16D68002D00D0CA61456A002D73
S1130FA000D0CC62002B11D0CA610A628A62CA6284
S1130FB08369022B01D14A628A61C168002902D186
S1130FC0406A002802D0FFF79DFFF2BD0020F2BD69
S1130FD080B5354801680122914301603348416B73
S1130FE0F82292010A4342630168314A0A430260CB
S1130FF0304800F097F801BD10B52B480168012274
S11310000A430260294C00F00DFE002804D0606BF6
S113101029490140616301E0284860632068284948
S113102001402160234800F0A1F810BD1F48016869
S1131030E022D2020A430260016B8022D2020A43F8
S113104002632048017880220A4302700179022257
S11310500A4302710120704780B51B480168026889
S11310601A480068090F491C484300900098110170
S1131070090F491CFFF726FF02BD80B5144801681B
S11310800268C807C00F401C124948431107490FA2
S1131090491CFFF717FF0090009802BD002070471D
S11310A000D00440FFF8FFFF00D00040048004405B
S11310B00000030400400240FFE1FFFFFFC1FFFF07
S11310C0FFFFF8F340210740448004404CA1FF1F78
S11310D064800440006CDC027047000030B4434379
S11310E051435D18010C0C00130C5C432D1980B2A4
S11310F0434392B251430024C918644124040B04AD
S1131100090C09195043C018694130BC70470000EC
S11311107047000001000020224A914200D00120C3
S11311207047000038B50400FFF7F4FF800000BFEB
S113113020A10958080C1C4A8218012013680125B3
S11311408D401D43156000211BA28B01E3181D680F
S113115005431D60535CDB06DB0E01259D40134BEC
S11311601D60491C0429F0D331BD000010B5FFF700
S1131170D1FF80000FA10A58100C0B4943181C68BA
S11311800120904084431C60002000BF0AA2135C2D
S1131190DB06DB0E01249C40054B1C60401C04282C
S11311A0F5D310BD004002400070044000E100E0AF
S11311B080E100E004003C101C1D1E1FC020000143
S11311C07749A5E077490A68904202D2D020C00549
S11311D070474A68904201D208687047CA689042D2
S11311E001D248687047CA68904201D28868704743
S11311F00020C0437047F8B500F087F86A4F80209C
S11312000005386000F02EF800F07FF8674C256880
S1131210B04E306800281AD0F0680021C9438842D3
S113122005D02800FFF7CEFFF16840182060902019
S11312300005386000F016F830690021C94388427F
S113124005D02800FFF7BEFF3169401820608020D8
S11312504004386000F006F83068002800D02560AB
S11312600020F2BDF8B5FA208000FFF702FD04006B
S11312700D00FFF7F8FC06000F0020002900FA22F9
S113128092000023FFF72AFF8019794104000D0022
S1131290FFF7E9FC8D4205D801D3844202D2FF2036
S11312A09A30F2BD9F480068C007F1D40020F2BD17
S11312B038B59D49E82252008A181368022B23D3BB
S11312C0374C23688025ED011D432560012811D189
S11312D01068002814D02168090E491C48431128BD
S11312E000D3102021680902090A401E00060843A1
S11312F0206005E0022803D1486CC0B200F087FDED
S113130020688A490140216031BDFF20801C884942
S11313100A6802430A600A680240FCD1704738B583
S1131320824C844D286820402860286803210143AA
S113133029600A20FFF7A9FC2868E14301432960DA
S11313402868032188432860286804402C6031BD44
S1131350794A7A4B00280AD0012812D0022813D0E7
S1131360032814D0042814D0102814D015E01878B9
S1131370002801D0002001E0FF2096300860002002
S11313807047D020C005F9E75868800AF6E710686E
S1131390F4E75068F2E75868F0E70420704700006B
S11313A000A0054080A1054008A0054000A105401B
S11313B0F0B589B0AC4800900068002800D0012046
S11313C0039000240025FA208000FFF752FC06AAAF
S11313D003C2039800280CD0FFF745FC04000D005D
S11313E000980068002106AA0CCAFFF777FE04AA39
S11313F003C201204C49896C88400290002001906E
S1131400AD4FAE4E039800280AD0FFF72CFC001B0A
S1131410A94104AA0CCA8B423ED301D882423BD3D1
S1131420FFF7CCFEFFF771FF34680098806800284E
S113143012D0009805690020C043854204D02000E2
S1131440FFF7C0FE40193060B02000053860FFF798
S113145009FF00283CD13460C02080043860FFF7C5
S113146001FF002834D1FFF7FEFB04000D0006A89D
S113147003C8FA2292000023FFF730FE04AA03C235
S1131480FFF7F1FB0B00021BAB4104A803C8994210
S113149005D801D3904202D2FF20983018E0F068BA
S11314A0F82149010140EBD0AA4800680190306E50
S11314B080214902014331661B48806CC0030198B6
S11314C0029902D581439DD101E001409AD10020C7
S11314D009B0F0BDE8ACFF1F30B583B00C009E49E5
S11314E0982212068018104A526B5200904204D27D
S11314F0D020C0050090486802E008680090886821
S1131500019000256846A90040586C4908602000F5
S113151002D0A047002803D16D1C022DF2D3002075
S11315203EBD00005CA1054014ABFF1FFFBFFFFFE1
S11315306CA1054000A00540D8ACFF1F14ADFF1FEF
S1131540F0B585B00C00A14902910968019180278A
S1131550FF04394300918118049106000025AE4828
S1131560C06D002806D00098B90A0143009101E03B
S1131570019836180498864271D20120FFF798FE2C
S11315804E4D2E60A448C06D002802D1FFF733FEF3
S113159004E0A2493000FFF79FFF2E600298006923
S11315A0002815D0FFF7B1FE0298406A039000218D
S11315B0C943884205D03000FFF704FE0399401860
S11315C02860A02000053C490860FFF74BFE2E6010
S11315D0FFF79BFEFFF7F2FD286E790001432966B1
S11315E0EFF3108072B6102122686A65241D491E2B
S11315F0FAD10321A965019940398908009A2E4B33
S11316001A607A0809E023686B6563686B65A368F0
S11316106B65E3686B651034091F012905DBEB6D0D
S11316201340F0D12B6E3B40F9D080F31088FFF7C4
S113163019FE0220FFF73CFE286E384002D0CC256C
S11316406D000CE07448C06D002802D1FFF7B0FEB5
S113165003E0C1493000FFF73FFF050088D0FFF7E2
S11316605EFE280005B0F0BDE0ACFF1FF1B5002020
S1131670D024E4050025684F08E00026002D05D09D
S1131680022D07D004D3032D06D006E07E6B04E0C0
S1131690BE6B02E0FE6B00E03E6C002E06D0AF484D
S11316A00460200000998847002803D1A4196D1C08
S11316B0042DE2D3F2BD000008A0054000A10540BE
S11316C0F8B504000120FFF7F3FDFFF794FDA44DE6
S11316D02868002821D0A14E0027FF43A869B842FA
S11316E005D02000FFF76EFDA96940183060FFF7B0
S11316F00CFEC020C0049B490860FFF7B3FD3460B2
S11317006868002801D0FFF776FDED69BD4204D07A
S11317102000FFF757FD40193060FFF7F6FD8020E9
S1131720800490490860FFF79DFD0220FFF7C0FD8B
S11317300020F2BD80B5FFF73BFE02BD10B58A481C
S1131740FFF794FF8948FFF791FF0400FFF7E7FDD7
S1131750200010BD00A2054080A10540F8B504009A
S11317600120FFF7A5FD7D4D2C60FFF744FD7C4E65
S11317707C4F3068002817D0B0690021C9438842E3
S113178005D02000FFF71EFDB16940182860FFF75F
S1131790BCFDC020C0043860FFF764FD2C60706895
S11317A0002801D0FFF727FDFFF7AFFDE020C004BC
S11317B03860FFF757FD0220FFF77AFDFFF7F8FDC9
S11317C00400FFF7ACFD2000F2BD0000D8ACFF1F01
S11317D070B5114EF16D00291AD0982109064118EF
S11317E04C08D020C0052018614D726B5200914204
S11317F006D2FFF7B3FF00280CD12868001907E0D0
S1131800FFF7ACFF002805D168680019716B401A16
S1131810FFF7A4FF70BD000014ABFF1FF711000019
S1131820F0B583B0CF49534ACA610A68E0239A43AA
S11318300A6002000C32926C002A03D00A688023EA
S113184013430B600126C84ABA235B00D3180193E3
S11318502023402405000C35ED6C002D34D00D6898
S113186025430D60D4256D0045192F68002F02D043
S11318700F681F430F60019F3F6B002F00D08E0C39
S11318800096AE68B702C02636013E40B446EE6804
S11318903604FC27BF03374066463743BC462E69EF
S11318A03706FC26B6053E4067463E43009F3E434E
S11318B0C068002808D06868002802D130004E0DA6
S11318C001E030008E0D06431032D06B032802D1A4
S11318D030009E0206430198806A002802D030003E
S11318E05E0206430198C06A002802D030001E023E
S11318F006434E62CD48D56DAD012C40956D6D010A
S11319002B402343146E2404E025ED0225401D439F
S1131910456080235B02D46C24041C400C620F24B9
S1131920019D2D6825409669360433402B4303609E
S1131930D069000223020340106A04401C4310686B
S11319400004C0239B0203402343CB60506BC0B20E
S113195000F05DFA0020FEBDB113000000A10540B7
S1131960E8ACFF1F08A00540C116000035170000B1
S113197084A1054000400080FEB50400FFF772FC1E
S1131980AB4800688021C9040143A94801602000D4
S1131990FFF7C5FAA74D002861D17348406BD021E9
S11319A0C9054118A44801606F4A926B89184160C7
S11319B06D4AD26B891881606B4A126C8918C160B8
S11319C09E4E9820000608187060D020C0050021A3
S11319D000912300343304211A681B1D002A02D00D
S11319E0076800978018491EF6D10098FFF797FC06
S11319F0706800280FD05C48C06D00280DD05A488C
S1131A00406B5949C96B884205D15748806B564988
S1131A10096C884201D00420FEBD00208849894A0F
S1131A200A6002224A6000224F4B96009B195B6FAA
S1131A30854E8700F351401C521C402AF4D3814840
S1131A40086001204860474800688021C9010143BB
S1131A50444801602000FFF7E3FE002805D07449E4
S1131A6009680D4072490D60FEBD3E480068774923
S1131A7001403C480160764D2869A90D0143296164
S1131A80BC204000205800283ED0D020C005009043
S1131A9020003430029004200190029800680299DA
S1131AA0091D029100282BD000992960009908187B
S1131AB00090BC20400020184068002820D0002658
S1131AC0B0002018BE21490047183868002817D0F4
S1131AD0FFF791FBFFF719FCFFF770FB38696865A6
S1131AE0002068656865686538681E498860FFF786
S1131AF0B9FBFFF75DFC002802D1761C042EDFD36E
S1131B000198401E0190C8D1E069002827D0D02652
S1131B10F6052000343000900427009800680099EE
S1131B20091D0091002818D02E603618FFF763FBBA
S1131B30FFF7EBFBFFF742FB20001C3040686865B1
S1131B40002068656865686520001C308068054968
S1131B508860FFF787FBFFF72BFC7F1EDDD1002099
S1131B60FEBD000000A0054014ABFF1FF0B583B01C
S1131B70002801D0810746D1304F002139700090F0
S1131B80FFF7CDF92A4801688022D2040A43026093
S1131B90304801688022D2010A4302600124446271
S1131BA001680902090A22060A4302602A49C1613E
S1131BB00E2101614161816101680C220A430260C6
S1131BC00168224A0A400260009800281DD1D025ED
S1131BD0ED050095286801900198FFF7A0FB1F4EC2
S1131BE02868B0420AD016481649016002224260B1
S1131BF01B4A02611B4A426101604460FFF78FFB8C
S1131C002868B04201D00420FEBD174D620200993D
S1131C10280000F035F92800FFF7AEFE002800D1B7
S1131C203C70FEBD054800787047000004A10540E3
S1131C3038800440FFFFFFFB80A1054014ADFF1F67
S1131C4000A30540F05AF05A10A30540FFBFFFFF60
S1131C5000A1054000A00540000800806B71636688
S1131C6013042008041C000014ABFF1FFEB506007B
S1131C70FFF7D8FF05006F4C002E69D16E4800684D
S1131C8060606E48806806696836307F317CC906BA
S1131C90CA0F69460A7268490968090F491C002D70
S1131CA001D0674A00E0674A0192C207D20F684632
S1131CB0037A01205840104001236B40184205D09C
S1131CC0A0204004FFF7FEF85F494CE00198FFF7BD
S1131CD0F9F85D490860707FC1430807000F401C94
S1131CE0009006460746002D03D0012000900326ED
S1131CF00EE06846007A002802D00120009006E039
S1131D0001983146FFF7DEF84E49884201D1022698
S1131D1037460098401E0007761E3106F022120551
S1131D200A4002437F1E3804F02109030140114395
S1131D304148016001980099FFF7C4F842490860DE
S1131D402A000121207800F011F801202070F7BD4D
S1131D50012E09D1002D07D100220021207800F0A6
S1131D6005F8606834490860F7BD0000884200D176
S1131D707047F8B5354810239F24354DFA26B60030
S1131D800027012921D102212973009703E000BF14
S1131D900099491C00910099B142F8D3302129706F
S1131DA0E9780C40002A01D1202100E040212143A0
S1131DB0E970A9791942FCD100970099814225D292
S1131DC000BF0099491C0091F7E700291ED1002AA1
S1131DD01CD134212970A9791942FCD02F730097A2
S1131DE003E000BF0099491C00910099B142F8D367
S1131DF004212970E9780C40EC70009703E000BFDF
S1131E000099491C009100998142F8D3F1BD114910
S1131E100A681202120A002802D0012804D007E03E
S1131E201000C022920402E01000802252040243F7
S1131E300A60704720AAFF1F4480044010A0FF1FBF
S1131E4000A24A04006CDC024CA1FF1FC05D00002C
S1131E500040064000A00540124207D08B0706D080
S1131E600B78491C0370401C521EF7D87047830737
S1131E7006D00B78491C0370401C521EF9D17047E0
S1131E8070B4103A03D378C9103A78C0FBD2530720
S1131E9001D318C918C001D508C908C0D20704D392
S1131EA00B880380891C801C002A01D50B780370E1
S1131EB070BC70470021C943C26E8A4205D1026FCB
S1131EC08A4202D1426F8A4201D0364900E0364943
S1131ED0C16270473EB504000D00684600F070F81A
S1131EE020000C302818001B051DA2686168A94257
S1131EF00BD28B18984208D2421A684600F066F852
S1131F006068A1684018421B2900684600F05EF82A
S1131F1002A9684600F085F802983EBDF8B5012490
S1131F2068460470214EB0680569E86A1E49884213
S1131F3034D00020694608702F006837B86800283C
S1131F402AD0796842428A4226D372681368994239
S1131F5004D352680818401E82420FD200F084F85D
S1131F60002819D07268203278681168884213D327
S1131F705168BA688018401E81420DD30C4928006C
S1131F806830FFF7A7FF696F884201D0094804E071
S1131F9068460470084800E00848E862684600782B
S1131FA0F2BD0000A2280000A328000010A0FF1F1B
S1131FB0C0A30000A1280000A0280000A42800005D
S1131FC00021C9430160002141607047F0B585B02C
S1131FD004000E001700684600F0C0F868460121AE
S1131FE0C172216801911B49009100218172018114
S1131FF0002F0FD000F0FFF8174D6946280000F0BD
S11320007BF83A003100280000F0AFF8286801900E
S113201000F0F7F8019820606068C019606005B0AE
S1132020F0BD38B504000D0020798007800F08D07A
S1132030694600220A6004210A1A69462000FFF753
S1132040C5FF2068286005480168054A0A40026007
S113205031BD0000B71DC104002003403C80044092
S1132060FFFFFBFF0120704780B5FFF7DBFD02BDDA
S113207010480068C103C80F70470F4800687047D4
S11320800D4908600D49896809694865704710B5AC
S113209082B000226B461A70084C0A00010020002E
S11320A020302469646CA04768460078002800D07A
S11320B0012016BD6C80044074A0FF1F10A0FF1FF8
S11320C010B54A7A92070B7A1B07C024A4051C405A
S11320D014438A7A93062343CA7A1206802464043A
S11320E022401A4382600B68436063001343836099
S11320F049680160826010BD70B584B0164A1368E7
S11321008024E4021C4314600322022300240D7B78
S1132110002D0D6800954D6801956D460DD14E7AE0
S1132120002E01D02B7200E02C720C7A002C00D00F
S113213002226A728A7AAA7207E02C720E7A002E40
S113214001D06B7200E06A72AC72C97AE9726946B6
S1132150FFF7B6FF7FBD00003C80044080B500BFA0
S113216013A11022FFF78CFE01BD03E00B7803706E
S1132170491C521E002A06D08B07F7D103E00B68D6
S11321800360091D121F042AF9D2002A03E00B7808
S11321900370491C521EFAD17047016880688000A0
S11321A0800F022801D3080C704788B270470000E2
S11321B021100000FFFF00000000000000000000EC
S11321C00160704772B60168491C016062B601681B
S11321D00029FCD10120704772B60168491E01E054
S11321E072B60021016062B6704772B600200A49D7
S11321F0086062B6704772B607480168491C0160FE
S1132200704705480168022900D2EAE70168491EBF
S1132210016070470000000038AAFF1F0020AF498A
S1132220C968C96808607047FEB5002600206A4680
S11322309670AA4CE7697D69002D75D0E168C9687C
S11322400A68012A5AD000230A000832091D3800FE
S11322506D68A847002805D0A149884202D0491CCE
S1132260884261D1E268D1688B68002B5CD002930C
S11322704868019000786B4618706846007800281A
S113228008D068460078132804DA9268C000101851
S1132290083800E0002008620127002822D00068E6
S11322A000281FD000A9491C20002030226992690F
S11322B09047050017D168464078002809D0E720E8
S11322C0400169460978491EC840384001D1854D0E
S11322D009E002990198E268D268126A126890478C
S11322E0002007E0B34D68460178280000F080FA2A
S11322F0280019D1E168C9680F60FEBD096A002988
S11323000DD04968080003D000A8801C884700E06D
S11323100020002803D0E168C9680E60FEBD69464C
S11323208978E268D2681160FEBD80B5017800202A
S113233000F05EFA6948C06941690969884702206A
S113234000F0B6FABFF34F8F9B489C490860BFF377
S11323504F8F00BFFDE780B514216048C068C06896
S11323600C3000F007FB01BD10B5040060680028C4
S113237002D0012803D005E000F0FEFB03E000F0EA
S1132380AFFD00E00420FFE7217800F031FA10BD32
S113239010B50400A1686068504A126852699047F9
S11323A0F2E710B50400FFF7D6FF4C48C068C068D8
S11323B061680161082101772178002000F018FA92
S11323C001F03CF810BD7CB5002401940094434D09
S11323D06B4601AA8168C9B24068C0B2AE68B668EB
S11323E0B047E968C9680C6100998A08019900F04E
S11323F007FA73BD10B50400A1686068C0B2374A1B
S11324009268D2689047BFE770B50400A568A748F2
S11324102E186068012809D1280001F009F9002864
S113242004D0300001F004F9002801D104250BE0A8
S11324302800FFF79BFB0500284E02D13068006896
S11324408047B068006945652178280000F0D0F91C
S113245070BD10B50400FFF77EFF2048C068C06857
S1132460A16801616168416104210177217800203C
S11324708BE710B50400FFF76EFF1848C068C0680A
S1132480A16801616168416103210177A1680020AD
S113249000F0CAF910BD38B50400104DE868C068F2
S11324A0002141610161007F042805D12868006989
S11324B08047002C00D10400E868C068017F200038
S11324C000F096F9C848844206D1E868C068007FE5
S11324D0082801D101F038F831BD000010A0FF1F19
S11324E01227000011270000F1B584B0BF4DE86841
S11324F0C06800240169002905D1049804700020F3
S1132500FFF7C9FF52E00121049A1170076940697D
S113251002900094E86901236A4601A94669766835
S1132520B047060004D0E8694169C968884732E0C9
S11325300098002801D1AC482EE0B84200D93800F8
S11325400090E868C068017F082910D10199C16032
S1132550009981610099019800F0B3FF0600C64814
S1132560864202D0093886420CD100260AE0019A3C
S1132570009902982B689B68984706000298009976
S11325804018029000983F1A05D0002E09D0E8693F
S11325904169C96888473000FFF77DFF04980470DB
S11325A004E0E868C068076102994161002005B051
S11325B0F0BD0000102700000400FA050CED00E057
S11325C0F1B58CB0894FF868C0680025016900290D
S11325D005D10C9805700020FFF75DFF59E001213B
S11325E00C9A1170016902914469C168027F029BCF
S11325F0212B00D320230193002915D0019A04A88C
S1132600FFF72AFC02980199401A0290F869012305
S1132610019A04A94669B668B047060002980028E2
S11326202CD0002E30D029E0019961180391032A9F
S113263007D104AA019920003B685B68984706000B
S113264012E0102A01D00C46DCE7467FFFF7D3FDE9
S11326500096019B04AA2100380020303C69E46BF9
S1132660A0470600FFF7CDFD039C002ECAD0F869F1
S11326700123002204A94469A468A0473000FFF79D
S11326800AFF0C98057004E0F868C06802990161BB
S1132690446100200DB0F0BD10B50400E268A168EB
S11326A06068524B1B68DB6898476DE6FF010000C9
S11326B07CB5060070680090B0680190F0687A4CB0
S11326C020600025494949681031002807D00A686C
S11326D0904203D34968491C814200D204250098E2
S11326E000F0A6FF002800D104253178280000F06E
S11326F07FF8002D13D100986060002000F0D8F816
S11327000198A0602068002803D080F3088880F333
S11327100988A06861688847002000F0C9F873BD83
S113272038B50400606800F083FF002801D104205C
S113273005E06568012000F0BBF8A068A84721788F
S113274000F056F831BD10B50400284A211D1000D0
S113275020301269D269904716E638B50400FFF7B5
S11327604AFD224DA36822000C3261682800203003
S11327702D696D6BA8470500FFF743FD21782800FC
S113278000F036F831BD30B583B00400684600214E
S1132790002206C0FFF72FFD144DA3686A46616846
S11327A0280020302D69AD6BA8470500FFF729FDEF
S11327B0A2686946280000F03CF837BD10B5040053
S11327C0FFF7C9FD0948C168C968A2680A6162685F
S11327D04A6110220A77E168C068C0684177A1683D
S11327E0002000F04BF810BD1227000010A0FF1FBE
S11327F010B584B06A46A02313700023537045E0DB
S113280030B589B06C46A723237000236370A3708E
S1132810551CE570019004E098000D58201885605F
S11328205B1C9342F8D31BE010B584B06A46A32323
S113283028E030B589B06C46AF2323700023637061
S1132840A3700225E5700190002808D19008801C2F
S1132850E070029220000C30FFF712FB00E00293BC
S11328601248C0690023E1788A00121D6946446950
S1132870A468A04709B030BD7D27000010B584B01E
S11328806A46B0231370012353700023937002230C
S1132890D370019002910548C06900230C22694657
S11328A04469A468A0471FBD6CA9FF1F10A0FF1FA7
S11328B070B505000024022D04D0002001F024FB93
S11328C0012D0ED0002605E0C16889680A0000D0F9
S11328D08847761C0D481821714340180168002967
S11328E0F2D1002D0DD1FFF786FCFEF7B6F901F009
S11328F087FB074804600120FFF7B8F9FEF77CFB6B
S113290062B6BFF36F8FBFF34F8F70BD000A000034
S113291008ED00E01206130A1A43130C1A4300BF11
S1132920094205D083070BD00270401C491EF9D11F
S1132930704700001206130A1A43130C1A4300BF0F
S1132940130030B414001500103902D310393CC000
S1132950FCD2490700D30CC000D504C0890002D3BF
S11329600280801C002900D5027030BC7047000032
S11329700022D5E70022E3E7EFF31080BB4948606B
S113298072B6704738B5BA4C65682A000421200035
S113299020302369DB6A98476A46012120002030F1
S11329A02369DB6A9847286800994018401E6860CC
S11329B0002032BDF8B504000D001600C14F796B3C
S11329C0484201002140621A5219534218404242BF
S11329D06B46380020303F697F6CB84700280AD125
S11329E068460078002801D06C20F2BD320029002E
S11329F0200001F02DFBF2BDF5B58BB00D0003AA4C
S1132A0000F038F904006AD1A808800004902F1A55
S1132A100020C04308900990002F06D03A000C987B
S1132A200499411808A8FFF717FAFFF7A5FF0B98B8
S1132A300499401807908E4D0498002809D0034645
S1132A400C9A0B99280020302C696469A047040073
S1132A500AD1002F08D0042308AA0799280020309F
S1132A602C696469A0470400804E706880F3108864
S1132A70002C34D16846007B002832D0FFF77CFF5D
S1132A800498002812D005A8029006A80190A8680E
S1132A900069006DC0B200900C9B049A0B99280049
S1132AA020302C69A46AA047040013D1002F11D050
S1132AB005A8029006A80190A8680069006DC0B23C
S1132AC0009008AB08220799280020302C69A46ADA
S1132AD0A0470400706880F31088002C01D0200007
S1132AE000E000200DB0F0BD70B588B005000C000A
S1132AF0002069468300CA50401C0828FAD3002CE1
S1132B000DD02026202C00D826006A46310028004B
S1132B10FFF772FF002803D1AD19A41BEFE70020D3
S1132B2008B070BDF8B507000E00FFF725FF504C44
S1132B30654B320039002000203025692D69A847F3
S1132B404A4D696881F31088002814D1A168096985
S1132B50096B00290FD0FFF70FFFA0680069036D10
S1132B60DBB232003900200020302469646AA047B7
S1132B70696881F31088F2BDF8B500203C4CA16867
S1132B8009690D0058358A696768296856423A68A8
S1132B90914228D1696891422ED1FFF7EDFE4A494E
S1132BA020002030226992689047304D696881F393
S1132BB01088002816D1A1680969096B00290FD073
S1132BC0FFF7DAFEA0680069016DC9B22000203069
S1132BD02269126A9047696881F31088002801D13C
S1132BE001212970F2BD8A4206D2314004D010007E
S1132BF0FFF798FF0028F5D169684A4216407242EF
S1132C0079688A42EED2491C891A1000FFF78AFFBC
S1132C10F2BD70B582B0150000222A70144C6B46C8
S1132C200A000100200020302669766CB047002895
S1132C3019D169460978297069460978002912D0A2
S1132C400A4D297800290ED1A0680069016DC9B226
S1132C50200020302269126A9047002801D06C209D
S1132C6076BD0121297076BD0000000028AAFF1F4F
S1132C7010A0FF1F70B582B005000E0014001148AB
S1132C8080680069006B002800D001202070FFF7E5
S1132C9073FE6A4670420321884341422800FFF7CD
S1132CA0B8FF0A494968002802D081F3108876BD2C
S1132CB081F3108868460078002801D00020207035
S1132CC0002076BD10A0FF1F6B66656B28AAFF1F4E
S1132CD038B505008E4844682034FEF7A3FF002869
S1132CE003D12072FF20963032BD69461020FEF7D2
S1132CF02FFB002826D10098002804D120686060AA
S1132D00C820400032BD8349884201D3481E009048
S1132D10206800994118491E616001212172002D2B
S1132D200FD17D4DA8606068E86069460320FEF716
S1132D300FFB0098286069460420FEF709FB009801
S1132D406860002032BD70B504000D001600FEF767
S1132D5069FF002802D1FF20963070BD320029009F
S1132D60200001F075F970BDF8B50D0014001E00C7
S1132D70FEF758FF0028694F02D1FF209630F2BDBC
S1132D80002C36D0387800280DD163480068401EE6
S1132D90284002D0FF209230F2BD0120387000207C
S1132DA0B8607D6002E0F868A8421DD1B8685A494D
S1132DB0096802198A4203D200942919F96001E0D2
S1132DC0091A0091009A310038181030FFF744F8BE
S1132DD0B86800994018B86000996D187618641A9C
S1132DE04D4909688842CBD100F02BF80028C7D0A0
S1132DF0F2BD0020F2BD7CB50C001600FEF712FFF8
S1132E00002802D1FF20963076BDB508AD00B60784
S1132E10B60F08E001AA0421200000F09AF8002867
S1132E20F2D1241D2D1F002DF4D1002E06D001AAAD
S1132E303100200000F08DF80028E5D100F001F801
S1132E4076BDF8B500250026344C207800281FD024
S1132E50A068314F3968884205D0FF22091A20182A
S1132E601030FFF757FD3A68210010316068FEF713
S1132E7067FB06002570A5600AD13A68210010316D
S1132E80606801F0FBF8002802D0FF209430F2BD06
S1132E903000F2BD70B50C001500FEF7C3FE00282B
S1132EA002D1FF20963070BD1B4846687042044032
S1132EB069420840454201E0AD1BA419002D0DD024
S1132EC02000FEF785FC002809D13100200000F025
S1132ED027F80028F0D0FF20943070BD002070BD8A
S1132EE080B5FEF79FFE002802D1FF20963002BD78
S1132EF0FEF724FC00280AD107498868C968091A22
S1132F00491C00F00DF8002801D0FF20943002BDC8
S1132F1010A0FF1F010000081CADFF1F2CADFF1FF8
S1132F200322D2434B421340594202400023DB4365
S1132F3001E0121D091F002904D010689842F8D03E
S1132F40012070470020704780B50020FFF7C0FEC5
S1132F5002BD80B513000A0001000020FFF704FF42
S1132F6002BD80B513000A0001000020FFF743FFF3
S1132F7002BD80B50A0001000020FFF78BFF02BDEF
S1132F8010B504006068A168814211D2401A6060E3
S1132F90A1669D482060E08A002805D021002831E0
S1132FA02000383001F07EF80120A060002010BD20
S1132FB0B84810BD10B504000021A74801F072F80C
S1132FC01022616A20002830FEF746FF22003832C2
S1132FD01021606A01F08CF8AF482060002010BD19
S1132FE010B50400606A4289A282C268921E6260BF
S1132FF04268AA4B9A4202D1017A022901DBA8480D
S113300010BD22003832102101F072F8A54820606A
S1133010002010BD10B582B00400606A4268A2614D
S11330200268D21EA26063689A4201D39E4816BD0C
S11330300289002A0CD0E2824189C91E2166B04966
S1133040216038342200102101F052F8002016BD0E
S1133050002069460870AB4A10002030126992695A
S1133060904768460078002801D0B64816BD200075
S1133070FFF786FF16BD10B50400A068401EA060CF
S1133080220038321021606A01F032F8206E401EAE
S1133090206601D1AC482060002010BD10B50400AA
S11330A0A068401EA060210028316B4800F0FAFFA0
S11330B0220038321021606A01F051F82000FFF735
S11330C05FFF10BD70B504000026A5686D1EA560E5
S11330D01022616A383000F0D1FF002802D1AD48D7
S11330E020600BE0E08A401EE082000404D06D1EE4
S11330F0A5600120A06601E09E26B601300070BDE7
S113310038B50400E08A002804D0626A1021100057
S113311001F025F87B4D626A216EE06D2B689B6897
S1133120984700281DD12069A168491E884204D30C
S1133130286800698047002813D11022616A2000A2
S11331401C30FEF743FF694620001C30FEF769FF80
S11331500098616E884201D0B54832BD2A4820608B
S1133160002032BD38B50400E08A002804D0626A29
S11331701021100000F0F3FF1022616A20001C30BF
S1133180FEF724FF5F4D626A1021E06D2B689B6897
S11331909847002820D1E06D1030E065206E10388B
S11331A02066112801D3A34814E0002801D0A248C6
S11331B010E028680069804700280DD16946200086
S11331C01C30FEF72EFF0098616E884201D09848AB
S11331D032BD0D482060002032BD10B504001C3003
S11331E0FEF7EEFE206E112801D3924800E09248CB
S11331F02060002010BD80B5426E016EC06D414B51
S11332001B68DB68984702BD99330000F8B50500D8
S11332105A20285A0105090FC00701D5082600E0E5
S11332200426EC6D042901D00420F2BDFEF7E3FF6F
S1133230344F330060352A002100380020303C69C7
S1133240646BA0470400FEF7DCFF002C01D02000D3
S1133250F2BD0020F2BD0000C4B1FF1F70B5040030
S1133260E56DB74E280000F0E3F9002810D02100E6
S11332701831606EA8470600012E03D12000FFF725
S11332807FFE70BD022E03D100F0D8F8002070BD7F
S1133290300070BD78270000E12F000053544D50DA
S11332A075270000153000007627000010B50200D5
S11332B05C325368011D4B600C689C4201D2A148EA
S11332C010BD137ADB0711D513684C69A3420DD1E5
S11332D05268002A0AD08A60498A002904D0010071
S11332E02831383000F0DEFE002010BD5A21415C48
S11332F0C90701D5B54810BDFFF742FE10BD000057
S11333007730000010A0FF1F02005A20115A042039
S11333108B0700D5704780B5CB070AD50905090F7F
S113332002D1FFF729FC02BD012909D1FFF7D8FD1D
S113333002BD5C3251681068A54A12685269904710
S113334002BD000081270000C530000038B5C46DFF
S1133350A04965185A3000880005000F012809D1DA
S1133360200000F065F9002804D0280000F060F97E
S1133370002801D1042032BD2000FEF7F7FB040031
S1133380934D02D1286800688047A86800694465A5
S1133390200032BD9D300000B0B505002F00583725
S11333A05A24E88A002804D06A6A1021100000F028
S11333B0D6FE3800696A1022FEF762FD0120395CEE
S11333C06418401C1028FAD33878E1B2884201D03E
S11333D08148B0BD594879780A2927D801A2525C9E
S11333E0974400BF340C141C4A24342C4A3840003F
S11333F02800FFF75BFFB0BD2800FFF7EEFEB0BD6D
S11334002800FFF7F8FEB0BD2800FFF727FFB0BD86
S11334102800FFF779FFB0BD0020B0BD2800FFF7FA
S113342095FFB0BD2800FFF7F1FEB0BD6930B0BD17
S11334307A270000653100000131000070B5674C47
S113344070212000FFF796FA65482060FEF7D3FE4E
S11334505F4C644D04232A0030212000203026696B
S1133460B66BB04704232A1D312120002030266981
S1133470B66BB04704232A000832322120002030E2
S11334802669B66BB04704232A000C32332120008E
S113349020302469A46BA047FEF7B3FE002000226D
S11334A0D24381006958914202D1401C0428F8D3C8
S11334B0042804D100200021002200230FC500208D
S11334C070BDF2B50700002400200025464E009987
S11334D08D4219D010203169401A0099491B0AE025
S11334E0002910D07A5D3369F2546D1C3269521C84
S11334F03261401E491E0028F2D1346100F005F803
S1133500002801D1E3E73948F2BD80B500203349F2
S1133510354A4A62CA68002A05D00B6993420BD027
S11335205B1C0B6102E08A6E002A03D10800096863
S1133530884702BD521E8A6602BD000012270000A1
S11335407F27000076270000F8B5214C2068006929
S11335508047002839D1214D5920285C042825D1E1
S11335602E005C363768380000F062F800281BD063
S11335700020FFF79DF95A352878800712D5706826
S113358070616168103100280CD00A68904203D33E
S11335904968491C814201D20420F2BD80F30888A5
S11335A080F30988B068B8471148F2BD08280BD1E8
S11335B00220FFF77DF9BFF34F8F0E480E490860D4
S11335C0BFF34F8F00BFFDE70C48F2BD7C2700001E
S11335D010A0FF1FFF010000792700003CB1FF1F6E
S11335E0B52F0000C4B1FF1FB0B1FF1F7D2700003D
S11335F07E2700000400FA050CED00E07B270000A4
S113360038B505000C000020FFF752F9A14804600A
S11336104560A0210902A04A1160016881F308886D
S113362081F30988406880470020FFF741F931BDE4
S113363010B582B0002806D00021C943884202D0C8
S11336409649884201D1002016BD00246A46022111
S113365000F04DFE002804D10098007A002800D024
S11336600124200016BDF0B589B08D4EB068006904
S1133670683001908B4F3D000AE00199097C0142BA
S113368005D0686981692800EA685268904718354E
S113369028680028F1D1002104AA03C202AA03C2A7
S11336A0FA208000FDF7E5FA06AA03C208210020EB
S11336B0FEF7EDFC002805D1A0200002416800912E
S11336C0046801E000240094FDF7E8FC00283AD1E6
S11336D00098FFF7ADFF002835D0FEF71FFC002847
S11336E031D0B068006986300078C00703D4210067
S11336F00098FFF785FF0198408A6B49884200D102
S11337006A4802AD002106AA0CCAFDF7E7FC03C50E
S1133710FDF7A9FA04AA03C202A803C8002901D12B
S1133720002810D0FDF79FFA04AA0CCA801A994108
S113373002AA0CCA994206D301D8904203D32100AD
S11337400098FFF75DFF3D0000E018352868002869
S1133750E2D00199097C0142F7D02800E9680968A0
S113376088470028F1D0002DD6D00AE00199097CC1
S1133770014205D0BD4203D03800F9688968884702
S1133780183738680028F1D1280009B0F0BD30B5E9
S113379083B0FEF72AFDFDF71BFC414C20002030CE
S11337A02169496888474248E06320002030216944
S11337B0096C8847A06800688047FDF727FAFEF780
S11337C051FC002830D0A0680069983005686A462A
S11337D00421200020302369DB6A984701AA0121D3
S11337E0200020302369DB6A98470020C0438542CB
S11337F015D00098A84212D2019940182D494018BA
S1133800A8420CD349422800FEF741FC002806D107
S11338102800FEF7ABF9FF219631884202D100203F
S1133820FEF7A4F9FEF72CFCFEF7E5FCFDF715FA0C
S1133830FEF7E7FC0020FEF719FAFDF7E7F9206828
S113384000688047A06840688047FFF70CFFE0618C
S11338500169002903D009680A0000D08847E0699B
S11338604169002903D009680A0000D08847E0684C
S11338700068804737BD38B5FFF789FF084CE56914
S1133880E06840688047E868C1680800F8D028000C
S11338908847F5E778A9FF1F08ED00E01104000050
S11338A010A0FF1F000A0000FFFF000088130000A3
S11338B068A0FF1F00FEFFFF7047000010B500283E
S11338C001D1042010BD904909680901090F0F298D
S11338D002D18022920203E00BA24900515A8A02CB
S11338E000210160426001228260D202C260874AE4
S11338F0930D1478A3404361D2788261016101621F
S11339004162002010BD00000800100018002000D3
S11339103000400060008000C0000001800100020F
S1133920000300040006000070B5002801D1042043
S113393070BDC46965680C2209A12800FEF78CFAE1
S1133940A14E6D1C3560A568142200BF07A1280094
S1133950FEF782FA6D1C756002202060002070BDA5
S11339608021017002780A42FCD0704701688022ED
S1133970D2000A430260BFF36F8FBFF34F8F7047CB
S113398038B5040001D1042032BD9048904A10603B
S1133990A048814201D06B2032BD44E0F8B58AB022
S11339A007000C00150001AA00F0E9FA059B2A00A3
S11339B02100380000F0CCFA060023D1019C0298C3
S11339C0009065196D1E28000099FDF77BFA002907
S11339D00AD028000099FDF775FA451C0098454364
S11339E06D1E01E000982418A54218D32002000A95
S11339F0902109050143764801600A988549884267
S1133A0003D06B2630000BB0F0BD380000F061FA33
S1133A1006003869010000D08047002EE2D038004B
S1133A2000F072FAEEE7200000F053FA05002000DF
S1133A3000F06AFA280032BDF1B588B00D00140018
S1133A401F00002C01D1042039E06A4600F097FAE7
S1133A50039B3A002900089800F07AFA06002ED158
S1133A60009D02E003982D183F1A002F23D02068F0
S1133A7057494860241D03992802000A042905D1E6
S1133A80C021C90401435248016009E0082907D153
S1133A9021684F4A9160241DE021C904014311604B
S1133AA0089800F016FA060008980069010000D092
S1133AB08047002ED6D0089800F026FA300009B0CE
S1133AC0F0BD70B5040001D0002A01D1042070BDFE
S1133AD03F480D062D0A9A4E2E4306601568456030
S1133AE0102902D01139032903D2082B01D15168BE
S1133AF08160200000F0EDF90500200000F004FAD8
S1133B00280070BD000000004C80044028000240E2
S1133B10F1B588B00D0014001F00002801D0002C5E
S1133B2001D104204EE06A4600F029FA0698401EAE
S1133B3005421FD138401DD1E919491E0EAA127839
S1133B40012A05D1002D10D1791E07290DD10DE0D0
S1133B500EAA1278002A08D1FF2907D9802212045C
S1133B60954202D3994A914200D30420002829D1D6
S1133B70174E0DE0652025E071682160241D06992B
S1133B80082902D1B1682160241D06996D187F1A95
S1133B90002F17D08E4801002940C02292040A4306
S1133BA032600EA90978090608430699042901D14F
S1133BB0B06002E0082900D17060089800F089F92B
S1133BC00028D9D009B0F0BD30AAFF1FFFFFFF4481
S1133BD004000240F8B50C0015001F00002801D0B5
S1133BE0002D01D10420F2BD7A4E2106090A7A4A39
S1133BF00A43326000F06DF900280AD17168296027
S1133C00102C02D0113C032C03D2082F01D1B1682F
S1133C106960F2BD6B66656B002801D0002901D193
S1133C20042070476D4800788207920F022A01D160
S1133C30002006E0C0220240802A01D1012000E0D9
S1133C40022008700020704710B5020001D000293E
S1133C5001D1042010BD0020604B1C78A407A40FE0
S1133C60022C1BD05E489B1C1860087800064C7818
S1133C7024040443887800022043CC7804435C6025
S1133C80087900064C79240404438879000220430F
S1133C90C97901439960100000F01BF910BD0000C0
S1133CA080B5002801D1042002BD0904744A85E0CE
S1133CB0F9B589B00C00160001AA00F060F9069B62
S1133CC032002100099800F043F9002836D101AAF6
S1133CD02100099800F053F9019C03980090604278
S1133CE000994A4202405542A54205D16D1803E0AD
S1133CF0F61BE41900982D18002E1ED0281B37003F
S1133D00864200D9070038000699FDF7DBF8210246
S1133D10090A802252040A432E490A600AA9097832
S1133D20090200040843FF2101432A48416009981D
S1133D3000F0CFF80028DBD000E000200BB0F0BD8D
S1133D40FFFF0043F1B588B00C0016001D0001D13F
S1133D50042031E06A4600F012F9079B320021008A
S1133D60089800F0F5F8002826D1009C194F05E0CA
S1133D700799761A8A089200AD186418002E1BD091
S1133D802002000A80218904014339600EA80078CA
S1133D9000060F49014379602868B860089800F06C
S1133DA098F80028E4D00F99002900D00C601099ED
S1133DB0002901D000220A6009B0F0BD0A43054978
S1133DC00A6000F086F802BD0000000000048000D4
S1133DD0FFFFFF0004000240FFFF00410200024019
S1133DE0FFFFFF45F9B585B00C001500002B01D18C
S1133DF0042043E0042300F0ABF8029000283CD1F7
S1133E00002600276019019005984069009001463A
S1133E10484201994A42024051422040081A0099FE
S1133E20FDF750F80390012509E03E490968203860
S1133E30CA43C2402A4000D07F1C0098241801982D
S1133E4084420CD220000099FDF73CF8202802D2CD
S1133E5034494968ECE7059989698842E5D3002F1C
S1133E6002D10698067008E00398874203D2022024
S1133E700699087001E006980570029807B0F0BD35
S1133E80FFFF0040002801D0002A01D10420704720
S1133E9009291CD801A35B5C9F4400BF0A121216B7
S1133EA01A1E22262A2EC06810600020704740681F
S1133EB0FAE78068F8E70068F6E70120F4E740696C
S1133EC0F2E78069F0E7006AEEE7406AECE76A200F
S1133ED0704710B5144C7021217000F02BF80028A5
S1133EE011D120001149096888472078810601D53D
S1133EF0672010BDC10601D5682010BDC00701D5DB
S1133F00692010BD002010BD38B50400200000F069
S1133F1011F80500002D03D1054804494968884774
S1133F2031BD0000180002400000024030AAFF1F0B
S1133F300C3000F0002801D104207047C06900282B
S1133F4004D00068022801D1002070476D2070471A
S1133F50002801D1042070475B1E194201D113408F
S1133F6001D0652070470368994204D3406818184B
S1133F708918884201D2662070470020704770B5C6
S1133F8005000E001400002D01D1042070BD202175
S1133F902000FEF7EFFC2868301A2060E8686060B3
S1133FA06868A968FCF78EFFA0600420E06008211F
S1133FB021616161A061E061002070BD80B5144899
S1133FC01449086014491548421A1548884203D018
S1133FD0002A01D0FDF740FF12481349091A01D005
S1133FE0FEF7C6FC11481249091A01D0FEF7C0FCBD
S1133FF010491148421A02D01048FDF72DFF01BDA7
S11340000020C0430E4908600E4908607047000054
S11340100000000008ED00E0E48F00005093000071
S113402000A0FF1F20A9FF1FF0B6FF1F00A4FF1F61
S113403020A9FF1F1C9400001C940000F0B6FF1F71
S113404080E100E080E200E080B500F0A7F902BD65
S113405080B513000A000100180003E080B51300C6
S11340600A001900FDF7F8FE002002BD10B50C008F
S1134070110001232200FCF7FBF910BD10B402E08B
S1134080401C491C521E002A09D00B7804789C421B
S1134090F6D002D20020C04302E0012000E000205C
S11340A010BC704770B50C004B4D002806D0102290
S11340B0010028001030FDF7CFFE06E02800103084
S11340C000210022002300264EC0002C05D010221F
S11340D021002800FDF7C0FE05E000200021002299
S11340E000230FC5103D1035280000F093F970BD72
S11340F0F0B585B006001500080904900024364F79
S113410028E0102231006846FDF7A6FE00983968C1
S11341104140009101987968414001910298B96841
S1134120414002910398F968414003916A4639007D
S11341301031684600F078F968460EC80EC7016869
S113414039600C3F102269462800FDF785FE1036C1
S11341501035641C04988442D3D305B0F0BDF0B587
S113416089B0040016000809049000251A4F2DE0B8
S11341701022210005A8FDF76FFE102221006846D9
S1134180FDF76AFE6A4639001031684600F05AF9B4
S11341900098396841400091019879684140019143
S11341A00298B968414002910398F968414003912B
S11341B005A80EC80EC7016839600C3F1022694675
S11341C03000FDF749FE103410366D1C049885420A
S11341D0CED309B0F0BD000000AAFF1F70B582B0B5
S11341E004000E001500002E01D1002076BD6A46A1
S11341F000F07DF8002806D12A0031002000009B41
S1134200DB685B68984776BD70B582B004000E0029
S11342101500002E01D1002076BD00F08DF8002895
S113422001D05B4876BD6A463100200000F05FF89B
S113423000280ED12A0031002000009BDB689B6817
S113424098475449002802D1009AD26800E000221D
S11342500A6076BD38B504000D006A4600F047F8E0
S1134260002815D10098C0684069002801D1662053
S113427032BD2900200000F05FF8002801D0444836
S113428032BD29002000009AD2685269904732BD9D
S1134290002DFCD1002032BD70B582B004000E00A8
S11342A01500002E01D1002076BD00F045F800284D
S11342B001D0374876BD6A463100200000F017F877
S11342C0002806D12A0031002000009BDB68DB684F
S11342D0984776BD38B5002400202E4D2968002962
S11342E004D009690A0001D088472C6032BD03005C
S11342F02748002A00D1704770B5274C64681460C1
S1134300002902D170BD103414601468002C12D03E
S11343102568002D05D16668002E02D1E668002EBE
S113432009D0AB42EFD365689D42ECD35918491EBE
S11343308D4200D3002070BD70B54118491E002283
S1134340154B9C682469D500641958345D681601BE
S1134350AD5966682468AC4201D1AE4205D08642AC
S113436003D3A14201D3012070BD521C022AE8D319
S1134370002070BD10B50848446804E000680100DE
S113438000D080471034E0680028F7D110BD000049
S1134390D827000048AAFF1F10A0FF1F1A48006872
S11343A00004000F401E0A282CD801A1095C8F4488
S11343B00A5210141A1E24282E5234008021890116
S11343C013E0802100E0C021C9010EE0802100E05B
S11343D0C021090209E0802100E0C021490204E073
S11343E08021890201E08021C90208484068103018
S11343F0890880229205521A02604A005118044A20
S113440089184160002070470070044010A0FF1F0D
S1134410FFFFFF1F10B50400FDF72AFE002802D09D
S1134420200000F033F810BD70B504000D00160034
S1134430FDF71EFE002804D032002900200000F001
S11344402CF870BD70B504000D001600FDF710FEC9
S1134450002804D032002900200000F039F870BD93
S113446070B50021FF2212028B00C3181C682506B8
S11344701600264036022E43250A15403543240EE5
S11344802C431C60491C0429EED370BD33480168D9
S1134490802292020A4302607047F8B504000F00BC
S11344A015002F4E0020C04330643800FFF7D8FFBA
S11344B02000FFF7D5FF2B48396801607968416017
S11344C0B9688160F968C1601020B060264919E0BC
S11344D0F8B504000F001500214E0020C0433064DD
S11344E03800FFF7BDFF2000FFF7BAFF1D48396809
S11344F0016079684160B9688160F968C160102021
S1134500B0601A49316030610003B16C0143B16499
S1134510174922680A6062680A60A2680A60E26851
S11345200A60B26C0240FCD00A692A600A696A60B7
S11345300A69AA600969E960B16C0843B06438008B
S1134540FFF78EFF2000FFF78BFFAC4202D028005C
S1134550FFF786FF00203061F1BD00003880044081
S113456000100540001205400D0210000C0210005E
S1134570E0170540012811D109488022D2050129FC
S113458006D108490A60016810220A430260704794
S113459005490A600168102291430160704700BF19
S11345A09040024000E100E080E100E0BFF34F8F63
S11345B0034804490860BFF34F8F00BFFDE700BF05
S11345C00400FA050CED00E0012811D1094880220D
S11345D09205012906D108490A60016880220A432C
S11345E00260704705490A600168802291430160B6
S11345F0704700BF5040024000E100E080E100E06D
S1134600084A8000105889014018016A002900D125
S1134610704780B54068002803D0034909680858EA
S1134620804701BD64A0FF1F08ED00E080B50021B4
S113463001E080B501210020FFF7E2FF01BD80B554
S11346400221F8E780B50321F5E7000030B5104AF0
S1134650104B00280ED0022801D00BD330BD0E48D9
S113466080246405012901D11C6000E01460016804
S1134670016030BD012400BF08A5285CC006C00E3F
S11346808440012901D11C6030BD146030BD00009C
S113469080E100E000E100E0104002400C0D250044
S11346A0002101807047F0B585B005000E001700A9
S11346B06846FDF753FD00206946C8722A880192B6
S11346C0114A009288720881002F11D0FDF793FDE2
S11346D00E4C69462000FDF70FFD3A003100200022
S11346E0FDF743FD2000FDF758FD0190FDF789FD1E
S11346F00198288005B0F0BD00880880044801684E
S1134700044A0A4002607047211000000020034060
S11347103C800440FFFFFBFF4F494068085C704742
S11347204D498A68002A08D04A6813780370521CDD
S11347304A608868401E8860704700210170704795
S11347405A2800D0704780B5434A01235354434943
S113475011615169884701BD80B53F49496988475E
S113476001BD0000F0B585B004003B4D696100BF98
S113477043A0616889004758684600F0F6F80126AE
S11347806846067246723648E86036482861022157
S11347906068A26890476946380000F099F8324989
S11347A0380000F021F901216068FFF7E3FE60683A
S11347B028188670002005B0F0BD000070B5040014
S11347C06068254D29188978002910D02CA1820011
S11347D08E580021FFF7CEFE300000F0D1F8002102
S11347E06068A2689047002061686918887070BD8D
S11347F019484160826081680029FCD1002070471B
S1134800F0B583B0070000BF1DA0B9004058009068
S113481004462C34206880210905084009D0216011
S113482007E001A8E9688847684600790099486369
S113483026602068084D8026B6043040F1D12068F7
S1134840310A084007D00098806B21603900C0B25B
S11348502A699047F3E7F7BD9CA0FF1F5947000062
S113486021470000414700000000020A80B50020F3
S1134870FFF7C6FF01BD80B50120FFF7C1FF01BDF1
S113488000C0024000D00240010C4A4A89180A685C
S11348900123834013430B6070470029016802D051
S11348A04E4A0A4002E08022D2010A430260704765
S11348B0002100BF04A28B00D358834202D0491CBC
S11348C00229F8D30800704700C0024000D002401B
S11348D038B505000C00FFF7EBFF00BF36A18000E0
S11348E00858FFF7D1FF01212800FFF7D6FF2868F9
S11348F00121014329602868400040082860286895
S113490037490140207B80070843A17B8906014386
S1134910607B00060843E17B0902C02292000A4042
S113492002432A6001220121280000F049F820787E
S113493080002818C1682B4A0A406168491ECB06CA
S1134940F021C90519401143227A92068023DB0421
S11349501A400A43617A49065B0819401143C16051
S1134960286801218843286031BD00210170082294
S1134970426001724172017341738173C173704764
S113498038B5050001242868204328600021280048
S1134990FFF783FF2800FFF78BFF00BF06A180000D
S11349A00858010C034A89180A688440A2430A6023
S11349B031BD0000007004400C003C100D003C10A0
S11349C010B503680C04FC2189032140012A02D19B
S11349D019430B0000E08B43036010BDFFBFFFFFD2
S11349E0FFCCFFBAFFFFFF808A0103D5026B064BA1
S11349F0134003638A0303D5026B044B1340036320
S1134A00026B114301637047FFFFFFFEFFFFFEFFD0
S1134A10010C164A89180A680123834013430B606A
S1134A207047010C114A89180A68012383409A438C
S1134A300A6070470029817803D080220A4382707B
S1134A4070474906490E817070470000002100BF7D
S1134A5004A28B00D358834202D0491C0229F8D304
S1134A600800704700600640007006400070044073
S1134A704022114202D083781A43827020221140CE
S1134A8002D081790A43827170470100C8788A791B
S1134A90520603D502008020C00110438979C9065B
S1134AA003D50100802040010843704738B5050054
S1134AB00C00FFF7CBFF264980000858FFF7A8FF3A
S1134AC0A07A002802D0022804D00DE0E08840003B
S1134AD0287009E0E0884000287020894000E871CF
S1134AE06879082101436971A878FD210140A07803
S1134AF0400008432178C9010143A97068796F21F6
S1134B0001402079000108436178C9010143DF2095
S1134B100840E17849010143697131BD10B500BF16
S1134B2004000021FFF786FF2000FFF78FFF00BF7E
S1134B3008A180000858FFF774FF10BD002181729E
S1134B4041708170C17001710121017070470000D2
S1134B50544B00000600341007003410002100BF3D
S1134B6004A28B00D358834202D0491C0329F8D3F2
S1134B7008007047004005400050054000600540B3
S1134B80F6B585B0040008680290049000200390F4
S1134B90694688800425069802996943FCF792F9CE
S1134BA086B2002E00D10126069829007143FCF735
S1134BB089F90299471A00910698711C6943FCF718
S1134BC081F90099081AB84201D20700761C0498AA
S1134BD0B84203D304970395684686806D1C212D43
S1134BE0D9D308466421FCF76DF9410008180499EB
S1134BF0884201D25E4867E02000FFF7AFFF00BFA4
S1134C003FA180000858010C5A4A89180A680123F8
S1134C10834013430B60A06857490140A16020689A
S1134C200399091F042903D201008020800208434C
S1134C30524901400398401E0006F82252050240E2
S1134C400A4368468088C004C00C10432060206872
S1134C504B4901402160A06810218843A060A068EE
S1134C6003218843A060A068059909790143A160E4
S1134C70206844490140059840794003802292010C
S1134C801040084320600598C0790004059989798B
S1134C900143E161A06988210143A161A069C021A8
S1134CA009020143A161A0680599097A002902D08B
S1134CB00100900108430599497A002902D00100B6
S1134CC050010843A060002007B0F0BD80B5C16961
S1134CD0FF2212020A40FAD141684902FCD50021A0
S1134CE08160FFF73BFF800005A10858010C214AB1
S1134CF089180A68012383409A430A6001BD0000B1
S1134D00140038101500381016003810E12149023B
S1134D1001600021017141718171C171017241729F
S1134D20704710B50A020368C024240214401C43CF
S1134D3004608369C024A40014401C438461826815
S1134D40FF2399431143816010BD41688069020CBF
S1134D50C32010400843704705E043681B02FCD59C
S1134D600B78C360491C13005A1E002BF5D1704701
S1134D702105000000700440FFFFF3FF00E0FFE0A6
S1134D80FFFFFFDFFFDFFFFFF8B515000126012459
S1134D904348006802000C320023DB43491E082903
S1134DA04DD801A77F5CBF4408244080804A80948A
S1134DB07C00696899420FD000290DD0D16801297F
S1134DC011DB4621415C01290DD1183009E06968E5
S1134DD0994201D0002901D10020F2BD1161167061
S1134DE01430FDF7F9F9002429E024212030FDF7DF
S1134DF0C1FD24E0A978002907D1E978002904D16C
S1134E002978012901D1567019E06A6829002030F7
S1134E10FDF722F8224800686968C16106731430FE
S1134E20FDF7DAF90BE0052409E000211430FDF761
S1134E30C7F900211A4800681830FDF7C1F92000AD
S1134E40F2BD38B50C000020012C0DD1144D28689A
S1134E50462281542423020020320221806800F07B
S1134E60C9F9296847310C7032BD0020002900D0EF
S1134E70704780B50A480068482142542423020040
S1134E8020320221806800F0B5F902BD04490860AF
S1134E900020704702490860002009688860704754
S1134EA03CAAFF1F10B513000120002B01D10320E1
S1134EB010BD00225A745A68002A06D014682200D1
S1134EC003D00A0001211800A04710BD10B513003B
S1134ED00120002B01D1032010BD00229A745A68CE
S1134EE0002A06D01468220003D00A000221180008
S1134EF0A04710BDF0B585B00600002501207168FB
S1134F008968327B4B79934247D30968002944D09E
S1134F10D20089180839002200E0521C0B789A420A
S1134F203BDA4B680C2454431B191C78032CF4D132
S1134F300021B77B00E0491C1A7A914206DA5A68CC
S1134F400C0112191478BC42F5D11500D97871738B
S1134F50002D22D0B560002402AF08E092480090F2
S1134F6001966A4602A9306800F06CFA641C29793B
S1134F708C4212DA00203871A000A968095CB9706B
S1134F80AA68121852883A80AA6810184078F870F3
S1134F90C8090128E2D18548E1E705B0F0BD38B57C
S1134FA004000120A16800290CD0002506E08868CF
S1134FB0A900415C206800F063FA6D1CA1680A79BD
S1134FC09542F4DB32BD000070B584B004001500D6
S1134FD00120002D01D0002C01D10320C0E00026C7
S1134FE0491E0529FAD802A2525C5200974400BF18
S1134FF0570307172D4226736674A674B0E06168E0
S11350000029FBD0217B2A788A42F7D0002902D0DC
S11350102000FFF7C4FF28782073A67311E06168AD
S11350200029EBD029880D00627B0904090E8A420D
S11350300AD1A17BEDB28D4206D02000FFF7AFFF6D
S1135040A5732000FFF756FF8AE061680029FBD0B2
S1135050A1680029F8D0A26811798E42F4DA29787F
S11350609268B300D25C914202D1206800F021FA28
S1135070761CF0E76168002972D0A16800296FD01E
S1135080A26811798E426BDA29789268B300D25CF7
S1135090914202D1206800F01AFA761CF0E72968E0
S11350A00A78D206D20E012A5AD10A79637B9A422F
S11350B056D120006A464B78012B0AD0022B10D01F
S11350C0032B16D0092B1DD00A2B38D00B2B3DD027
S11350D045E04988090A11722968498851720321F7
S11350E01CE022000F32042163681B6898470F34C8
S11350F006E022001032042163681B6898471034CC
S11351006C602DE04988090A117229684988517236
S1135110297B00290AD0A9680191092163681B68C9
S11351209847009969600199A96019E0696800913C
S1135130A9680191062163681B68984710E04988B3
S1135140090AE1732A68921C072104E04988217442
S113515022001032082163681B68984700E005208C
S113516004B070BDF8B50C00170000250021104AEA
S113517014234B43D6183268002A04D0491C012951
S1135180F5DB0220F2BD310000F053FA00280AD109
S11351903068002801D10320F2BD74603573FF200C
S11351A0B0733E600020F2BDCD4E0000A54E00005D
S11351B0A4A6FF1F10B5040001D1032010BDFFF702
S11351C0EEFE0021216061602173A17310BD10B552
S11351D0002801D1032010BD0400607C002801D008
S11351E0022010BD206800F011F9002801D101212E
S11351F0617410BD10B5002801D1032010BD040056
S1135200A07C002801D0022010BD206800F006F91F
S1135210002801D10121A17410BD000010B50400C3
S113522000F020FB002020608D34207000F024FB6F
S1135230002010BD38B5002801D1032032BD4468D8
S1135240002C08D000680D0602D5A468A04732BD22
S1135250E468A04732BD062032BD80B5002801D1E4
S1135260032002BD4368002B03D000685B699847A4
S113527002BD062002BD3EB505000A7A13071B0FC6
S1135280D4090120102A19D100220B212800FFF78C
S1135290E4FF28008C300221817000240470002077
S11352A0C1006918CC600C61401C1028F8D300229E
S11352B001212800AB68984700203EBD082B11D27D
S11352C05A001443E200AB18DA68002A0AD00868CE
S11352D0009048680190487A694608721A69280063
S11352E0DB6898473EBD80B5002901D0002801D174
S11352F0032002BD8268002A01D1012002BDFFF70C
S1135300BAFF02BDF7B50500002A01D10320FEBD96
S113531000F0A8FA2A4E37008C373068002806D0EF
S113532079788D4203D100F0A7FA012540E00224E8
S1135330002803D000F0A0FA022539E07D7000F0C7
S11353409BFA0198B0607D70002000213970CA007A
S1135350B218D0601061491C1029F8D3012D18D857
S11353608AA07060174800280ED0174800280BD078
S11353701648002808D01648002805D015480028EB
S113538002D01548002809D13000FFF747FF072055
S1135390FEBD3000FFF742FF0620FEBD32003100A3
S11353A0280000F0B5FC050004D0300000F01CF823
S11353B02800FEBDBC70029806600020FEBD0000FF
S11353C014A6FF1F115D0000895D0000C35D00008D
S11353D0355E0000EF5E0000415F000080B50022F2
S11353E00021FFF73AFF02BD10B5040001D10320EC
S11353F010BD6168002904D02068496888470020EE
S113540060602000FFF70AFF002010BD10B50C07F4
S1135410240F80212143FFF70DFF10BD80B509073C
S1135420090FFFF707FF02BD80B5002801D1032053
S113543002BD4268002A03D000681269904702BD89
S1135440062002BD10B5002801D1032010BD00299B
S113545014D0002A12D08B781C07240FDB09082CE7
S11354600CD264002343DB00C3181468DC60526868
S11354701A610A000221FFF7F0FE10BD042010BDDE
S113548073B504000D072D0FCE09002C01D10320A4
S113549076BD01AA0321FFF7E0FE082D07D26900BB
S11354A00E43F10061180022CA600A6176BD04202F
S11354B076BD02B5694609780907090F082904D29F
S11354C06A460421FFF7C9FE02BD042002BD02B5ED
S11354D0694609780907090F082904D26A46052193
S11354E0FFF7BBFE02BD042002BD000058B5030057
S11354F00120002A01D1042052BD1C008C34891ED5
S113550006291AD801A6765CB74400BF080C1E22EF
S1135510101626000C210DE00D210BE00020A178CF
S113552001E000202178117052BD062102E007211C
S113553000E009211800FFF790FE52BD10B50300EA
S113554001201C008C34032906D0062906D0072923
S113555009D0092915D010BD0E2113E0002A14D05A
S11355600020117808E0A178032907D0002A0CD084
S11355700020117821700321A17010BD22000821A0
S113558000E00A211800FFF768FE10BD115D00005D
S1135590895D0000C35D0000355E0000EF5E000021
S11355A0415F000070B504000025002600F05AF9A0
S11355B086481421714340180168002906D0817C73
S11355C08C4203D10560456085742EE0761C012E63
S11355D0EEDB13E070B505000C00002600F042F984
S11355E07A481421714340180168002903D0817C52
S11355F08D4200D118E0761C012EF1DB00F03CF95D
S1135600042070BD70B505000C00002600F02AF9D6
S11356106E4814217143401801688D4200D103E0A3
S1135620761C012EF4DBE9E7206000F025F9002068
S113563070BD70B505000C00002600F013F9634836
S11356401421714340180168002904D0817C8D42E3
S113565001D10068E8E7761C012EF0DBCEE70000FC
S1135660F7B50125002A04D06946FFF7CBFF0028CF
S113567001D00420FEBD002405E0521CD2B2032A4E
S113568007D3641CE4B200984168087A844219DAAA
S1135690002208680C236343C01800BF65A31601E9
S11356A09B191E7B87683F79BE42E6D1029A694600
S11356B0097940689B689847052804D00028E0D100
S11356C00025DEE72800FEBD70B582B004000D00A1
S11356D016006946FFF796FF002811D1012D08D165
S11356E00099200000F0DFFF009A02212000FFF75C
S11356F0B7FF320029002000009B5B685B68984775
S113570076BD0000F4B506000C000125002A04D083
S1135710002C02D06068002801D10420F2BD00F002
S1135720A1F800202949142242438A181368002B47
S113573002D0927C964210D0401C0128F3DB00205A
S1135740142242438F183A68002A09D0401C0128C9
S1135750F6DB00F091F8022513E000F08DF810E07C
S1135760BE7400F089F87C603A0019493000FFF7F4
S1135770C9FD050007D03868FFF736FE3000FFF793
S113578011FF2800F2BD002517E0002478680068A6
S11357900C216943411800BF26A0220183188868A0
S11357A000791A7B904203D10A1D30001B68984788
S11357B0641C032CEAD36D1CEDB27868007A854230
S11357C0E3DB3868009908600020F2BD00A6FF1FE3
S11357D0C9560000F8B507006946FFF7FBFE040050
S11357E026D1002516E000260098406800680C21A8
S11357F0694340180FA132018918826812790B7B22
S11358009A4202D1406849688847761C032EEBD33C
S11358106D1CEDB200984068007A8542E3DB009885
S11358200068FFF7E1FD040002D13800FFF7BAFE7B
S11358302000F2BD65510000B5510000C94F0000C1
S113584001000000CD800000C1810000DD81000066
S11358500300000000000000000000000000000041
S1135860000000000A480178002900D172B60178CE
S1135870491C01707047000005480178002904D0D4
S1135880491E0170C9B2002900D162B670470000F8
S11358901CA9FF1FF8B5040017000D006E003E435D
S11358A0FFF7E0FF30012018C26A8021C9011143CB
S11358B0C162FA07D20E2B07DB0D08256B4E676811
S11358C037401F431743490A29403943009F4F601B
S11358D0C06A61680E4033431A43410A0D401543C0
S11358E00699890589094009402210400843882106
S11358F001432960FFF7C0FF09E180B5C16A0822AE
S11359004B0A1340C3180C330362002383624262C0
S1135910574A0A40802189011143C162082100913C
S1135920036A00220021FFF7B5FF01BDF8B5011D90
S1135930FF224B6888331A704B6894331C78022515
S113594025431D70002300244D6898352C70474D65
S11359502607F60D00960E682E40009F37433B60E5
S11359600F682F40009E3E43082737433B600F6873
S11359702F40009E3E43102737433B600F682F4063
S1135980009E3E43182737433B6066018619F36245
S11359906600012737433E018619F3624E68A7006B
S11359A0F619C0363370641C082CD1D390246400DB
S11359B0001903704C6894342578FD262E40267017
S11359C04C688C34227089224C6884342270437071
S11359D0486894300178DF220A400270F1BDF1B5C5
S11359E082B00C8888780207120FC30950001D008A
S11359F0054390000090C448C978012904D1411C92
S1135A008C420DD304000BE0412C00D340240299B6
S1135A108968009E8919C0310E78012737430F70B9
S1135A2002992D014919CE6AB84D3540CD62AD0AAF
S1135A30AD0220402843C8620D4C0440CC62CF48DC
S1135A402040C862002B01D0042000E00820029905
S1135A508968009C0919C0310C78204308701343ED
S1135A6002D10298FFF749FF0020FEBD00FEFFFFB0
S1135A70FFF7FFFF70B504000E07360F7000CD0965
S1135A800543200000F033FAA068B1004018C0308C
S1135A900021017028012018C16A890A8902C162A3
S1135AA0002070BDF8B504000807000FC9094300C1
S1135AB00A001A431201A218D56AB04B2B40D362D4
S1135AC0AF4D1D40D56200230E0145013543666884
S1135AD0760A76022E43DD072D0F35432E687607AE
S1135AE005D5D66AB605B609082737432F605B1C6F
S1135AF0022BE9D3A2688300D218C0321378FD25A3
S1135B001D401570014302D12000FFF7F6FEA06886
S1135B1094300178DF220A4002700020F2BDF0B513
S1135B2089B00500AA688032107C0F23070901217F
S1135B30C60801243440029484080120204008242B
S1135B4014706A68540A64027A012243029C240194
S1135B501443C20022431468A201920D0092002251
S1135B60A40823400D2B01D1012600E000267C006F
S1135B70029B23431B061B0DEC18E36A9B0B0B4093
S1135B805CD0002E03D090235B00EB18D8700298F1
S1135B9000283ED0A06A00994018A062616A081AE1
S1135BA00190E16A802000014840E06280214901BF
S1135BB04140E1620198002804D000988905890DCC
S1135BC088421ED2A06A0690206A0590E16A4F4876
S1135BD00840E06200998005800D81421ED1002FAB
S1135BE01CD1606A902149006918C978C9006918F4
S1135BF0498A884212D2002300212868FFF706FC54
S1135C001CE0019B226A80213943280000F0D9F866
S1135C1014E00098384313D10692059205A8467201
S1135C200299C9013943017205A92868FFF75BFB92
S1135C30A86894300178DF220A40027009B0F0BDF0
S1135C40E06A430B19401FD169684B0A5B02790172
S1135C501943400A08231840084340680490206A06
S1135C60A16A4018039004980399884209D000203F
S1135C7004E00499095C039B1954401C0099884270
S1135C80F7D3902040002A54A06A00994018A062DB
S1135C90616A081A0190002F10D1002E0ED08021C5
S1135CA0280000F024F9E86A802109010143E9622F
S1135CB0E86B802109010143E96304E0E06A802183
S1135CC009014140E162E16A802040014840E0620C
S1135CD0616A002907D00199002904D00099800540
S1135CE0800D814208D2A06A0690206A0590E06A7D
S1135CF006490140E16291E7019B226A39002800CC
S1135D0000F098F89AE70000FF030000FFBFFFFFD0
S1135D1070B582B00D001600694600BF19A2136861
S1135D200B60002827D1824C9121490060540098CF
S1135D30A060891C6118E161FF218030017000229C
S1135D400121200000F0FCF87A486060000AA16894
S1135D509C3108706068000CA168B03108706068FC
S1135D60000EA168B43108702000FFF7DFFD346035
S1135D702560002076BD062076BD0000FFFBFFFFF6
S1135D80FFF7FFFF00200740002801D103207047E0
S1135D90FF21826880321170816884310A78002280
S1135DA00A70836898331A70816894310A70806825
S1135DB08021490040180178C0220A430270002063
S1135DC07047F1B582B01C0001200F270F230B4050
S1135DD05B0003430126029D1B01ED18EB6A9B0B3C
S1135DE0184006D1A8622A626C62E86A7203024310
S1135DF0EA62E86A8005800DA04200D204000F40E8
S1135E000298FF212231405C002809D10094286ABD
S1135E10A96A4318012239000298FFF73BFD0600E6
S1135E20A86A044304D1002F02D10298FFF765FD4C
S1135E303000FEBDF7B582B01C000F27084638407D
S1135E40410001200126029A09015518E96A890BCB
S1135E50014003D1A962049929626C62E96A420390
S1135E600A43EA62E96A8905890DA14200D20C005D
S1135E700499AA6A891801910299902252008918FA
S1135E80029AD269002A12D00A78002A0FD1412C32
S1135E900DD20322144202D1019B134207D0EA6AB5
S1135EA0254B1340EB62029AD2690192087068464E
S1135EB0007B07404878002807D10094019B00220A
S1135EC039000298FFF7E6FC0600002C0CD1002FE5
S1135ED00AD1E96A802040014840E862174901403C
S1135EE0E9620298FFF709FD300005B0F0BD10B576
S1135EF084B00A07D30ECA091A4312018218D36A5E
S1135F005C04E40F10D00023DB430193136A009375
S1135F106B46197200215972D16A084B0B40D36247
S1135F2069460068FFF7DFF9002004B010BD0000E7
S1135F30B8A6FF1F00A4FF1FFFDFFFFFFFBFFFFF87
S1135F40F8B5040001230120002C01D10320F2BD87
S1135F50042580260C29FAD801A77F5C7F00BF4462
S1135F60061F2E353C666D7182A0A0899C0000201E
S1135F70A1681A028854A068017F294202D0017FD7
S1135F800E430677A0688421490040180178102246
S1135F900A430270A068943001780B4303707AE0DE
S1135FA0A068017F294203D0017F4906490E017789
S1135FB0A0688421490040180178EF2234E0002AC7
S1135FC06FD011002000FFF70AFDF2BD002A68D04F
S1135FD011782000FFF74EFDF2BD002A61D0117840
S1135FE00E07360FCD0970002F0007432000FFF77E
S1135FF07EFF38012118CA6A8020C0001043C8629D
S11360006168490A490272010A4329011143420A9B
S113601008231A400A43800580098C21014311603A
S1136020A06894300178DF220A40027033E0002A2D
S113603037D011782000FFF735FDF2BD002A30D0AB
S1136040138028E0002A2CD011780B071B0F082B93
S113605027D25800C909014308012018C06A400525
S1136060C10F518017E0002A1BD01078A168983125
S1136070087010E0002529003143C9B22000FFF761
S1136080F9FCE9B22000FFF7F5FC6D1C082DF2D3F2
S11360902000FFF74BFC0020F2BD002A01D00020B5
S11360A01070F2BD002800D1704770B584B0046848
S11360B0A06880300678300702D52000FFF72FFD56
S11360C00125F0070FD5FF2122316554A1688031E5
S11360D00D7000200090694610220A7201904872E7
S11360E02068FFF700F98020064212D0A1688031B1
S11360F00870E06B800A284003D1E06A800A0540FA
S113610007D080212000FFF7CDFC00212000FFF7FD
S1136110C9FCA068AE21490040180178002900D0CC
S113612001707FBDFEB582B00600052401AA0621D8
S11361303068FFF7DBF968460079012805D0684626
S11361400079002801D0052030E00298007802256B
S11361501F210327084208D132001032042130687D
S1136160FFF7C4F90400308A18E000221F2303401B
S1136170012B02D10024328212E00140022911D104
S11361800298808869460870684642806A460521FC
S11361903068FFF7ABF9040068464088074037824F
S11361A004980560103603980660200005B0F0BD21
S11361B070B582B006000C00052500206946087001
S11361C000AA521C06213068FFF790F9684640780F
S11361D0012805D068464078002801D0052076BD06
S11361E06078032802D101206946087020781F21B5
S11361F0084208D1608801282BD16A4610213068F2
S1136200FFF762FA24E00140022922D160880028C5
S11362101FD1A0880F2210420ED10240C1091143A0
S113622030686A461278002A03D0C9B2FFF741F9F0
S113623002E0C9B2FFF74BF93068694609780029D2
S113624002D0221D052101E0221D0621FFF708FAD4
S11362500500280076BD38B505000C006A46062105
S11362602868FFF743F96846007803280BD0012813
S113627003D0022801D0052032BD60886946087029
S11362806A4607210BE0002207212868FFF756F928
S1136290002807D10120694608706A46062128684B
S11362A0FFF74CF932BDFCB585B007000D0005249D
S11362B06E88300A009001AA06213868FFF716F9A3
S11362C068460079012805D0002803D0022801D0AF
S11362D0052037E0E88803900098012802D102AA3B
S11362E0092124E002A80099022903D1067202AA16
S11362F00A211CE0032905D18672A988018102AA1A
S11363000B2114E0212904D1A988017202AA0C21CD
S11363100DE0222904D1A988017202AA0D2106E008
S1136320232908D10672A988417202AA0E2138686D
S1136330FFF7CAF9040002980599086003980699C2
S11363400860200007B0F0BD70B582B004001500ED
S11363501E006A4606212068FFF7C8F868460078E0
S1136360012805D068460078002801D0052076BDB4
S113637001203060200010302860220010321121EA
S11363802068FFF7A1F976BD38B505000C006A4610
S113639006212868FFF7AAF868460078012805D086
S11363A068460078002801D0052032BD00206946E7
S11363B008706A4606212868FFF7C0F8608800283C
S11363C007D10120694608706A4606212868FFF74C
S11363D0B5F8A21C03212868FFF742F9A21C072183
S11363E02868FFF771F932BDF8B504000D001600F6
S11363F01F006A4606212068FFF778F8684600788F
S1136400002801D00520F2BD0120386020001030A2
S11364103060287920822200103212212068FFF790
S113642053F9F2BD38B504000D006A460621206810
S1136430FFF75CF868460078002801D0052032BDDB
S1136440A8880002A9780143218222001032042185
S11364502068FFF705F92200103208212068FFF7B1
S113646033F932BDF8B504000D0016001F006A466A
S113647006212068FFF73AF868460078002801D022
S11364800520F2BDA888208222001032082120684D
S1136490FFF72CF81034346002213960F2BD7CB56A
S11364A006000D0001208024052A10D129786022DD
S11364B0114207D0214205D1E988002902D0002BDE
S11364C000D10020C1013000FEF7F3FF76BDE9885A
S11364D007980268914200D2016003680698026836
S11364E000213000FEF792FF002808D129782142CC
S11364F005D00023002200213000FEF78FFF76BD77
S1136500F5B589B00F000025039504950524786836
S11365100021C943884213D00A98002810D00646A7
S1136520083602AA06210998FEF7E0FF4020397ACE
S1136530002975D07968082902D13968002901D168
S11365400520AEE04A8872808A88B280CA88F280C8
S11365504A78727009783170602319420CD100BFF7
S113656065A091004558280054D004AB03AA31001B
S11365700A98A84704004DE00122F388002B29D093
S11365800B0627D48B060BD5069505A80273059632
S1136590F088079005AA01210998FFF761F80CE03B
S11365A0014237D0069505A802730596F088079036
S11365B005AA0F210998FFF787F8040007980490AB
S11365C00698039026D1F388039A00210998FEF7D0
S11365D025FF66E08B060BD5069505A80273059684
S11365E0F088079005AA01210998FFF739F80CE013
S11365F001420FD0069505A802730596F08807900E
S113660005AA0F210998FFF75FF804000798049082
S11366100698039004A8019003A80090002339E091
S11366206946097A032909D104AB03AA31000A98FF
S113663031A47578AD006459A04730E07968002929
S11366402ED0F18800292BD031780A0628D48A0666
S11366500CD53868069005A80573059678680790E8
S113666005AA01210998FEF7FBFF0DE001420CD0B9
S11366703868069005A8057305967868079005AAFA
S11366800F210998FFF720F8040004A8019003A83B
S113669000900123220031000998FFF700FF040055
S11366A020000BB0F0BDF0B585B007001148009094
S11366B0019102AC012020710026E6708020A070B8
S11366C0402020806A4602A93800FEF7BBFE050080
S11366D00ED1A6706A4602A93800FEF7B3FE050083
S11366E005D080213800FEF7CBFE280000E0002012
S11366F005B0F0BD0165000025610000B161000036
S113670000000000B16100000000000057620000BA
S1136710A7620000000000004963000089630000D4
S1136720E9630000256400006564000000298178A5
S113673003D080220A43827070474906490E817053
S1136740704780B5002000F0ABF801BD80B5012092
S113675000F0A6F801BD6D494068085C70476B49BC
S11367608A68002A08D04A6813780370521C4A6069
S11367708868401E8860704700210170704780B5AA
S113678062494969884701BD5A2800D0704780B5DD
S11367905E4A012353545E4911615169884701BD22
S11367A0F0B585B00400594E716102216068A26899
S11367B090476068009000BF59A00099890045582F
S11367C001A8FEF7BBF901A81021C18051498968CD
S11367D0096979310978FF2900D0C18001A928000D
S11367E0FEF764F901212800FFF7A0FF40212800EB
S11367F0FEF73EF9FAF730FC2F00FA218900FAF788
S113680061FB01004448FAF75DFB002100E0110040
S11368104A1C13004343322BF9D30125002905D127
S1136820FF22F632904204D2012102E0202900D353
S11368301F21B879F02202401143B9710121009857
S1136840FDF7C2FE3548306160683018857000205D
S113685005B0F0BD70B5040060682C4D2918897826
S1136860002914D02EA182008E580021FDF7ACFE21
S113687000213000FFF75AFF3000FEF74FF90021E6
S11368806068A2689047002061686918887070BDCC
S11368901E484160826081680029FCD10020704755
S11368A070B582B0040000BF1DA0A10045582800A7
S11368B0FEF7EBF812220240EA7050210140102941
S11368C012D01021114AEF23460612D54007A878AA
S11368D00BD50143A9700020694608706846D16849
S11368E0884768460078287173BD0340AB702879E7
S11368F073BDAE780E4203D0C007ECD5A878F4E798
S1136900287921001269904773BD0000B4A0FF1FCD
S11369107F67000010A0FF1F40420F00896700003E
S113692000600640007006407FB504006668694652
S11369303000FAF7F9F8002836D100BF42A0B100C0
S1136940455801A8FEF7E2F9009801903000FAF7E3
S113695094FB020001A92800FEF712F9002820D1B7
S113696002213000A268904701213000FDF76EFE3D
S1136970802189032800FEF7D4F9A8688021C90280
S11369800143A960A868802109030143A9602A4C36
S11369905A2061688847A620616888470120A0556D
S11369A003E03000FAF7A2F8002004B070BD10B57F
S11369B004002148416001216068A2689047606832
S11369C0FAF794F8002010BD38B5040065681A4839
S11369D0405D002809D000212800FDF737FE00BFE4
S11369E019A0A9004058FEF771F92800FAF798F8A1
S11369F000212800A268904731BD000080B500BF87
S1136A0011A3406880001858FEF7A6F9002002BDC3
S1136A1010B50A4C01E010B5094C2000FEF795F9B9
S1136A20800204D5E068C0B203494968884710BDB4
S1136A3010B5044CF1E7000040AAFF1F00400540D8
S1136A4000500540006005400040054000500540EE
S1136A5000600540F8B50B00110001250120C04C71
S1136A6026685B1E062B30D801A7FF5CBF4400BF1D
S1136A7008162E384A5A5800002926D00868400AB9
S1136A8000F0C8F805E000291FD00868400A00F0AB
S1136A9081F8002819D02168BD4A8D54F2BD00291F
S1136AA013D058368E60F2BD00290ED058368E6051
S1136AB00868400A00F0AEF8F2BDC003086080091F
S1136AC048600D748860C8600020F2BD00207047E3
S1136AD070B5A34C2060583000F0CEF9256828002A
S1136AE0583000F04BFB06008421C90054352800BF
S1136AF0FBF740FF20688C21C90046500021416506
S1136B00002070BD96490860002009680865704738
S1136B10F8B50124924F3868B149405C002805D18A
S1136B20FCF78CFC3868AE4A845444653868AD4937
S1136B30405C00282DD002253968A94A8D5400F004
S1136B4011F90600F7D03868A5494018C168002932
S1136B5006D10178022903D1032000F02EF900E0C8
S1136B604470A148864214D038689E4940180021D8
S1136B7001709E498E4201D1C574F1BD62398E42C5
S1136B8002D1C574032002E00321C174002000F087
S1136B9014F9F1BD70B582B005000C0084204000EA
S1136BA0854235D36E4E3068914941180A78002ADF
S1136BB00ED18878002801D00F2076BD6946A068E0
S1136BC000F0B0F8002823D0009800F0E3F803E0C8
S1136BD08849405885421BD13068864941184B6822
S1136BE06268934200D21A008E68B6188E609B1AAF
S1136BF04B606D1C0D60002B02D100217C4BC154F5
S1136C00A16896239B00C018FBF726F9FFF780FFC5
S1136C10002076BDF8B507000C006168A068FBF79A
S1136C20A7FE00BF26A000E00C304168002906D072
S1136C300268BA42F8D18268A068FBF70DF9484DA2
S1136C4028688C21C900401832A6002F08D0FF21E3
S1136C50891C7F1A0ED07F1F20D07F1E22D02CE0EB
S1136C605520A168FF2252008854AA20A168521C12
S1136C70885422E0A4687B316118006800F086FA29
S1136C8028688E21C900405C8000305800F076FAF4
S1136C90CE214900611800F079FA0EE0A06800F0F6
S1136CA0EBF80AE0007C80003558280000F066FA12
S1136CB002002900A068FBF7CFF80020F2BD000015
S1136CC000000000B00600003600000001000000D3
S1136CD0E80600000E00000001010000F8060000B4
S1136CE0A0010000030100009808000060000000FB
S1136CF00401000048090000A00000000501000094
S1136D00F80800004D000000000000000000000032
S1136D1000000000800600008806000098060000BD
S1136D20A406000030B505000C00143000F038FA59
S1136D30A649884211D12800343000F031FAA44920
S1136D4088420AD1287E012807D11C35280000F08A
S1136D5027FA00012060012030BD002030BD000072
S1136D6050AAFF1F80B5244800689A494218136846
S1136D70802189008B4203D2190001D11A4802BD37
S1136D805B1A1360962292008018FCF79AFB02BDEE
S1136D905904000010B518490B688F495C1801218B
S1136DA0217061700022A270E17022718D24E400D0
S1136DB01B195A601860197210BD10B50E49096884
S1136DC0854A8C180122227000236370A070E3703E
S1136DD023718D20C000081843600360027210BD47
S1136DE05C0400005D0400007D270000742700009F
S1136DF05B0400006404000050AAFF1F30B5302279
S1136E000270782242700022827200BF7BA31C248D
S1136E109500641B0D00E5402C07240F1C5D8518AC
S1136E20AC70521C082AF2D330BD70B504000D00BA
S1136E300026002D0ED028000A21FAF743F830313D
S1136E40A15528000A21FAF73DF80500761C002D0B
S1136E50F1D102E0302020700126A0190021017038
S1136E60401E05E00178227802702170401E641CE7
S1136E708442F7D370BD0000F1B5C0B057488068B4
S1136E800669306814907A20375A5548874200D1F1
S1136E90544F5548016826A8FFF7B0FF103626ACBA
S1136EA0316820000B30FFF7A9FF30687168411882
S1136EB0491E20001630FFF7A1FF71692000213020
S1136EC0FFF79CFF7069B1694118491E20002C30FE
S1136ED0FFF794FFB16C20003730FFF78FFFF16CA0
S1136EE020004230FFF78AFF316D20004D30FFF75C
S1136EF085FF716D20005830FFF780FF716815A879
S1136F00FFF793FF15ADB16828000B30FFF78DFF35
S1136F10316928001630FFF788FFB1692800213055
S1136F20FFF783FF390028002C30FFF77EFF2F483E
S1136F30016828003730FFF778FF2DA12DA2B06D2E
S1136F402D4B984201D1130000E00B00306A002859
S1136F5000D0110028003730139028002C301290F4
S1136F60119310920F91200058300E9020004D3054
S1136F700D90200042300C90200037300B90200000
S1136F802C300A90200021300990280021300890EC
S1136F902800163007900B35069520001630059012
S1136FA00B34049415A8039026A8029014A8007822
S1136FB0019014A84078009014A88378C27800BF88
S1136FC013A1409800F0F8F841B0F0BD53544D506F
S1136FD07367746C6C0400005A04000010A0FF1F57
S1136FE0FFFF000088130000248004404CA1FF1F11
S1136FF06E6F0000796573006B63666730313233FE
S113700034353637383961626364656600000000E0
S11370104B696E6574697320426F6F746C6F616441
S1137020657220256325642E25642E25640D0A0DC2
S11370300A53797374656D206465766963652049C4
S1137040443A2025730D0A466C6173682073697A8B
S1137050653A2025732062797465730D0A466C6164
S113706073682072616E67653A2025732D25730D50
S11370700A466C61736820736563746F7220736968
S11370807A653A2025732062797465730D0A466C1B
S113709061736820626C6F636B733A2025730D0A09
S11370A052414D2073697A653A20257320627974C0
S11370B065730D0A52414D2072616E67653A202551
S11370C0732D25730D0A526573657276656420729B
S11370D06567696F6E20303A2025732D25730D0A7C
S11370E0526573657276656420726567696F6E2098
S11370F0313A2025732D25730D0A56657269667918
S1137100207772697465733A2025730D0A436865A4
S1137110636B207265736572766564207265676956
S11371206F6E733A2025730D0A426F6F7420636F7C
S11371306E6669672070726573656E743A20257394
S11371400D0A5065726970686572616C20646574BB
S1137150656374696F6E2074696D656F75743A2028
S11371602573206D730D0A43505520636C6F636B58
S11371703A20257320487A0D0A000000010000E03F
S1137180491C0A78002AFBD1081A70478446087003
S1137190000A4870000A8870000AC8706046704788
S11371A0C3788278417800781B021A4309021204DA
S11371B008431043704700000CB41CB5040004A835
S11371C00190009401AB0A006946084878441C30D9
S11371D000F01BF80021009A1170002801D40098D7
S11371E0001B02B0019910BC03B008470F9DFFFFBC
S11371F070B5060008001400002B05D01D0021788E
S1137200B047641C6D1EFAD170BDFDB586B00C008C
S113721009E00123079A21000698FFF7E9FF04001B
S11372200798401C079007980078002801D109B0FE
S1137230F0BD2528EDD107984678801C0790252EAF
S113724000D195E0582E69D0632E0ED0642E1AD04A
S1137250692E18D06F2E61D0702E68D0732E70D026
S1137260752E5BD0782E59D0DDE708980068089910
S113727008600168001D089A1060C9B22000069ACF
S113728090470400CFE708980068089908600568EB
S1137290001D08990860002D04D52D212000069AB0
S11372A09047040064266F2E01D1082106E02021B6
S11372B03143782901D00A2100E0102101910B21EA
S11372C000912F00642E03D1002D01D578420700D0
S11372D0009D6D1E009538000199F9F7F3FD3031DA
S11372E0C9B23A2902DB30005138091802A84519FD
S11372F0297038000199F9F7E5FD070002D00098DC
S11373000128E5DA20000B21009A8C1AB9D02978DB
S1137310069A90476D1C641EF9D1B2E7089800687C
S1137320089908600568001D08990860BBE708987B
S11373300068089908600568001D089908607826A7
S1137340B1E708980068089908600568001D089965
S113735008602800FFF712FF01002000002990D0E8
S11373600C002978069A90476D1C641EF9D188E7B1
S1137370252183E710B5A048806804696834342166
S11373809E48FAF784FE002808D134229B49200045
S1137390FAF776FD2068B849884204D0FF223421E8
S11373A02000FBF7C7FAF9F797FE002010BDF8B5E7
S11373B0914DA86804694B20E0700220A07000265B
S11373C0667026705021E1710127A77160712671E2
S11373D05420E072A772667226722763A74860631E
S11373E0220010320421280020302B69DB6A9847E0
S11373F0220014320121280020302B69DB6A9847CF
S1137400220018320021280020302B69DB6A9847BB
S113741022001C320221280020302B69DB6A9847A5
S1137420220020320321280020302B69DB6A984790
S1137430220044320521280020302B69DB6A98475A
S1137440220048320621280020302B69DB6A984745
S113745022004C320721280020302B69DB6A984730
S1137460A16948420021C943854A53420340C91ACD
S1137470844A1040A065E1658348206683486066BD
S11374806869E66007E07822A35C0B4202D0E268F8
S11374901143E160761C1821714341580029F2D14F
S11374A07B48016821644168E1638068A06368687F
S11374B010300168616241680068081A401CA062CB
S11374C02000FAF7F7FC2765FAF7D7FD606500207E
S11374D0F2BD0000F4B582B00A001E00464B996864
S11374E0096904246B4D401E18285ED801A73F5C2F
S11374F0BF4400BF1A2C3034383C484CB650546258
S1137500B64044686E868C9094989CA0A400002E8B
S113751000D034600298002800D001600020FEBD35
S11375200C31F4E71031F2E71431F0E71831EEE7EB
S11375302031ECE72431EAE72831E8E73431E6E7A3
S11375402C31E4E73031E2E7D86941694969884779
S113755028602900DBE710245831D8E74E4800683A
S1137560F6E76946180020301A6992699047684620
S113757000780028ECD00120EAE70C243831C6E773
S11375804431C4E74831C2E74C31C0E75031BEE76B
S11375905431BCE70831BAE79C310D00100000F00B
S11375A02FF80028BBD11824D3E73C48FEBD0200C5
S11375B01148806803693A48521E072A18D9093AC3
S11375C00BD0521E012A13D9D21E032A10D9083A0D
S11375D009D0521E022A0BD90CE0002901D001293E
S11375E009D1196302E0032905D219650020704707
S11375F0401E7047801E704710A0FF1FC0A30000EC
S11376007AB588B0274C00E00834002C05D06168B6
S1137610002902D021688142F6D16268100001D1AC
S1137620042026E06946002090470098002820D1D5
S113763002AD2D1D029001260020019001A9300009
S113764062689047002808D1019828600298711E4A
S113765001228A400243029201E0002028602D1D8D
S1137660761C062EE8D3182202A90898FAF708FC1B
S113767000200AB070BD00006B636667FFEF010075
S11376801C9400000000000000A0FF1FEFC6FF1FB5
S11376905880044010ABFF1F248004403C280000A5
S11376A03E2800001006000010B50100A34A100097
S11376B0883003685C1C0460D218203211700168A1
S11376C08906890E016010BD0020704780B500F066
S11376D0C6F802BDFAB583B01700002901D0002F07
S11376E001D104202CE000263E60944C2000903010
S11376F00090467000F0B3F8002821D101AD02E0FB
S1137700A22000F082F820212000FBF733F968461C
S1137710027C210001A800F013F9002801D03E608A
S11377200EE0210001A800F089F9A9888142E7D17F
S1137730012000990870039804606888386000206C
S113774005B0F0BDF2B582B015001F00002944D089
S1137750212D42D200F083F800284DD1774C20002F
S1137760913000260178002900D006702000603096
S113777000905A2000990870A42000994870002FA6
S113778002D0A52000994870200062300570290AB3
S11377904170002D05D02A00029920006630FAF7C6
S11377A05BFB21006631009800F048F964342070D6
S11377B0000A6070A91D009800F064F800281BD12D
S11377C001AC01A800F028F9002815D16078A1289F
S11377D011D0A22805D0A32801D00420FEBD8848DA
S11377E0FEBD00984188891D00F04CF8002803D1A3
S11377F06078A228E5D00020FEBD82480121817076
S11378000021017070472020704780B569465A22D4
S11378100A70487001207C4908700221684600F013
S113782031F802BD10B582B0040076480178427880
S11378300A408078024210D1684600BF8DA10A88B0
S1137840028002226946200023695B689847082267
S113785089A1200023695B6898476C4816BD80B5F0
S1137860684800210278002A02D00170A12004E0B7
S11378708278002A04D08170A320FFF7C6FF02BDDE
S1137880002002BD80B503006148C0690A001900E8
S113789003695B68984702BDF3B585B01500002401
S11378A0F9F7E1F96A4603C2FA208000454328004B
S11378B0F9F7DFF902AA03C2564D0FE06868296898
S11378C088420ED01D4908182030007805990855C3
S11378D0641C6868401C8006800E686006988442B8
S11378E029D0F9F7C0F902000B00684603C81F004D
S11378F0161A8F41684603C88B420DD801D38242C1
S11379000AD2684603C8C043C94312184B41002039
S1137910521C434116001F0002A803C8002901D1CC
S11379200028CBD002A803C88F42C7D301D886420F
S1137930C4D3052000E0002007B0F0BDD4B1FF1F80
S113794070B582B004000D00160000F065F8002840
S113795055D16078A62804D12D48C069FFF762FF8D
S113796076BDA421002E00D0A521884201D001209B
S113797076BD142202216846FFF78EFF6946098806
S1137980A170090AE170002839D1A078E1780906CC
S1137990090C0843212801DB202004E0A078E178C9
S11379A00906090C0843A070000AE07014220221A1
S11379B06846FFF771FF694609882171090A6171F8
S11379C000281CD1A178E2781206120C114316D0BB
S11379D0A178E0780006000C01432800FAF7C8FFFC
S11379E0A078E1780906090C0843A178E278120628
S11379F0120C11430A2242432800FFF74DFF76BDC3
S1137A001227000064B2FF1F65B2FF1F1327000096
S1137A1010A0FF1F5CB2FF1F10B50400002201215B
S1137A202000FFF739FF002807D120785A28F5D124
S1137A300A220121601CFFF72FFF10BD30B583B06F
S1137A4004000D006846FCF72BFE04222100684662
S1137A50FCF729FEA278E0780006000C0243290016
S1137A606846FCF720FE01A96846FCF745FE684617
S1137A7080883EBD5AA70000000201500000AAEA17
S1137A8000480047D97A000000480047D97A00002E
S1137A9000480047D97A000000480047D97A00001E
S1137AA000480047D97A000000480047D97A00000E
S1137AB000480047D97A000000480047D97A0000FE
S1137AC000480047D97A000000480047D97A0000EE
S1137AD000480047D97A000000480047D97A0000DE
S1137AE004480549C1810549C181E9214900018052
S1137AF0704700BF0020054020C5000028D90000C1
S1137B0005207047087A002805D11B4808604C20DE
S1137B1048600020704705207047052070471748CB
S1137B2008601220486000207047087A002805D1B8
S1137B3013480860402048600020704705207047C3
S1137B4010B5887A0F4A002802D1106852680EE0F6
S1137B5092680B891489A34202D1042800DA01D166
S1137B60052010BD83001068C0585268D2584A607E
S1137B700860002010BD0000B8A1FF1F04A2FF1F71
S1137B8018A2FF1F5CA3FF1F002101604160FB30AE
S1137B90417001700020704738B504005830811CD2
S1137BA000250D708D72CD721430210030310A68B9
S1137BB002600A79D2094275C879002830D00328B6
S1137BC02AD0042838D012281ED0152840D01A28CC
S1137BD03AD01B284CD01D2842D01E2828D0232858
S1137BE03AD025282CD0282812D02A281CD02F2877
S1137BF03AD055282CD05A2826D09E2820D0A82800
S1137C0006D0AA2810D037E0200000F0A9FD32BD2C
S1137C10200000F0CDFD32BD200000F093FD32BD08
S1137C20200000F027FE32BD200000F0F0FD32BD40
S1137C30200000F013FF32BD200000F0EEFE32BD44
S1137C40200000F066FE32BD200000F023FE32BDAD
S1137C50200000F039FE32BD200000F073FE32BD7A
S1137C60200000F028FF32BD200000F005FE32BDE8
S1137C70200000F022FF32BD200000F041FFEC3470
S1137C8025706570E570A5702572E57132BDF0B59B
S1137C9085B00F00140001216A461173796826002B
S1137CA0ED3600250022D243914217D130780028C6
S1137CB026D060680068002822D03720205C28285D
S1137CC001D0A8281CD101953868029000956A4615
S1137CD00121200063681B68984711E0221D926807
S1137CE08A4202D3511A221D9160B179012909D126
S1137CF0B571012070703570317B2068FDF7D9FBB8
S1137D00012050E03178002903D179680D2900D190
S1137D1038683178002932D060680068002840D083
S1137D207868019038680290201DC0680090372060
S1137D30205C282801D0A82805D16A46012120000A
S1137D4063681B689847201D806800280ED0201D9A
S1137D50C06879684018211DC860200000F050FBFD
S1137D6069460873201D806800281AD135700D23D8
S1137D7022004832317B2068FDF748FB11E0796826
S1137D800D290ED10068824988420AD10120F07081
S1137D901F2322002832717B2068FDF73FFB01205E
S1137DA030726846007B05B0F0BDF2B584B01400B3
S1137DB0002669460E70049841682000343025007E
S1137DC0EC350022D243914217D16978002927D09B
S1137DD061680968002923D0C0782A2801D0AA281C
S1137DE01ED10296049800680390019601AA02210C
S1137DF0200063681B68984712E0221D92688A423B
S1137E0002D3511A221D91600127297A012909D12F
S1137E102E72EF702E706E72A97B2068FDF749FBFD
S1137E200020B3E0297800292BD0049949680291F5
S1137E30049909680391211DC968019161680B685F
S1137E40190018D0C0782A2801D0AA2803D101AA81
S1137E50022120009847201D806800280FD0201D93
S1137E60C068049949684018211DC860200000F0CA
S1137E70FEFA69460870201D8068002867D12E70BC
S1137E806CE02979002972D0049949681F296ED1C0
S1137E90211D496A824A914269D14178F0221142F6
S1137EA065D18178E022114261D142782B7B5B1C41
S1137EB09A425CDA00295AD0112958DA6E72211DCF
S1137EC08E6033494161C661211D896A81612E71C9
S1137ED0211DC96A221DD16280220378134203D175
S1137EE0002902D0012100E000212970007810420D
S1137EF005D0201DC06A002802D0012000E0002027
S1137F0068706878002804D0A878002801D001207F
S1137F103CE02000FFF740FE6946087068460078A0
S1137F20052812D12878012805D1E878002800D145
S1137F302F722E7007E06878012804D1A8780028F1
S1137F4000D1EF716E700220E872287800281BD1EE
S1137F506878002818D1E879002815D10D2322006B
S1137F604832697B2068FDF751FAAF720CE0A97BB7
S1137F702068FDF79EFA697B2068FDF79AFA2E7156
S1137F80EF70AF70EF726F716846007805B0F0BDA6
S1137F9055534253F0B587B00600002400940120E5
S1137FA069460873706880683500EC35297C42792D
S1137FB08A4225D30068002822D0C9004018083816
S1137FC0002100E0491C0278914219DA42680C232E
S1137FD04B43D2181378082BF4D10020EF7B00E038
S1137FE0401C117A884206DA51680301C9180B78DB
S1137FF0BB42F5D10091D07868740098002801D173
S113800001204AE0B06000270BE0A973694804909E
S1138010059604AA01A93068FDF714FA69460873A5
S11380207F1C00980079874219DA01A90C71B80005
S113803000998968095C01AA9170009A92681218E3
S113804052886B469A80009A92681018407801AA68
S1138050D070C8090128D8D169735748D7E72C7064
S11380606C70EC70AC702C72EC7101202871F460AF
S11380706C71AC71EC72687A012803D1A97B306809
S1138080FDF7D2F91F2332002832A97B3068FDF7AF
S1138090C5F9012068726846007B07B0F0BD000096
S11380A05553424338B504000120A16800290CD07F
S11380B0002506E08868A900415C2068FDF7E0F926
S11380C06D1CA1680A799542F4DB32BDF4B588B021
S11380D00D003A4C2168002901D0022067E02100FC
S11380E0FDF7A7FA060003D02000FFF74DFD58E086
S11380F02068002804D12000FFF746FD032056E045
S113810065602000F53000900025C571FF200099BE
S11381108871019402AA0521204663681B68984768
S11381200600039900293ED0029800283BD002A8FB
S1138130007C009AD070029A6261A161401E009A8C
S1138140D0700498206205986062E561220058327C
S1138150702010700A20D0719570958163695B1E40
S1138160FF2424021F0620001840000238431F0A7F
S113817027400743180E3843D0620B0627000F40F0
S11381803F021F430B0A1C403C43090E2143116369
S11381909063D16300990D70009845700198089917
S11381A00860300003E02000FFF7EEFC012009B076
S11381B0F0BD0000AB7D00008F7C00001CA8FF1FF9
S11381C038B5040001D1032032BDFFF76BFF050071
S11381D02000FFF7D9FC280032BD0000F4B582B0BE
S11381E005000124002A01D0002D01D10320FEBD89
S11381F02E00EE360027491E05290AD801A04900A1
S1138200405A87447A010A000E002E005C00B60032
S1138210B773F3E068680028FBD0B07B1178814223
S1138220F7D0002802D02800FFF73CFF029800781E
S1138230B07310E068680028EBD010880700F17B69
S11382400004000E81420BD1707BFFB2874207D03D
S11382502800FFF727FF77732800FFF79BFE040031
S1138260CCE068680028FBD0281D40680028F7D0BF
S11382700097281D4068009902799142F0DA02992A
S113828009788068009A9200805C814212D130782B
S1138290002805D12868FDF70CF90400012030708E
S11382A07078002806D1029801782868FDF701F952
S11382B0040037700098401C0090DAE768680028D2
S11382C0CED0281D40680028CAD0F0780128C7D035
S11382D000971CE0029909788068009A9200805CFB
S11382E0814211D13078012804D12868FDF7EFF8D4
S11382F0040037707078012806D102980178286844
S1138300FDF7E5F8040037700098401C0090281D24
S11383104068009902799142DCDB707A032801D02D
S1138320022812D13079012812D0307A012803D1E1
S1138330F17A2868FDF778F80D232A004832F17A9B
S11383402868FDF763F8377277723079012855D1C0
S11383503078002852D1707800284FD13771307AA4
S1138360012803D1F17A2868FDF75EF81F232A005B
S11383702832317B2868FDF751F8377277723DE077
S113838010680178CA06D20E012A37D10279F37B2C
S11383909A4233D180224378FE2B02D0FF2B15D092
S11383A02CE08388F67BB34227D14388002B24D169
S11383B0C088022821DA11421FD0F835029845609E
S11383C002980068C0880299886017E08388F47B6B
S11383D0A34212D14388002B0FD1C08800280CD1AE
S11383E011420AD12800FFF75DFE2800FFF7D2FDF5
S11383F00400F7700120307100E005242000FEBD68
S113840070B584B004000025002620690090206A1D
S11384103249884200D3481E0190E06801998142A4
S113842000D20800019002956A4604212000636886
S11384301B6898472000ED3021696269A3695A439B
S1138440914207D2019B029A017B2068FCF7DEFF70
S1138450060009E0857101214170057002218172D5
S1138460017B2068FDF725F8300004B070BD70B5BD
S113847084B004000025002620690090606A174932
S1138480884200D3481E0190E0680199814200D2DD
S11384900800019002956A460321200063681B6866
S11384A098472000EC3021696269A3695A439142DC
S11384B007D2019B029A817B2068FCF7AFFF06007C
S11384C009E005720121C17005700221C172817B2E
S11384D02068FCF7EEFF300004B070BD010001001D
S11384E010B5536884696343C360126883695A434F
S11384F00261012902D1FFF783FF10BDFFF7B7FF27
S113850010BD0000F0B583B0040000260020250053
S11385106C352100583101912968002905D126655F
S11385206968002900D000E103E10198801C0090F3
S11385302700EF37687D0028686878D0002809D1C3
S113854021656B68AA68B97A2068FCF75FFF002888
S11385501BD19FE0AA7D002A5ED088421DD2081A52
S11385602065019828300078012806D10C352A00AE
S113857001212000FFF7B4FF05E06B68AA68B97A0F
S11385802068FCF743FF0028E3D001205434207016
S1138590032000990870112085E08142266514D1DA
S11385A0019828300078012806D10C352A000121D1
S11385B02000FFF795FF05E06B68AA68B97A206888
S11385C0FCF724FF00281FD1B3E028680199283163
S11385D0097801290FD1A169F8F774FC2861296889
S11385E0A2695043081A20650C352A000121200095
S11385F0FFF776FF05E00300AA68B97A2068FCF764
S113860005FF002800D18BE001215434217003219F
S1138610009A1170112192E021650023AA68B97AA9
S11386202068FCF7F3FE0220543420703DE000285B
S113863009D1F97A2068FCF73CFF286820650120FD
S1138640543420700CE0AA7D002A0BD0F97A2068FB
S1138650FCF72FFF28682065022054342070012085
S1138660387022E0884222D2081A20650198283006
S11386700078012806D10C352A0000212000FFF7DC
S11386802FFF05E06B68AA68F97A2068FCF7C6FE3C
S1138690002802D15434267007E00120543420709D
S11386A0032000990870009988720520FEBD81425C
S11386B0266517D1019828300078012806D10C3599
S11386C02A0000212000FFF70BFF05E06B68AA6871
S11386D0F97A2068FCF7A2FE00282AD0012154343C
S11386E0217029E02B68019828300078012810D1E6
S11386F01800A169F8F7E6FB28612968A2695043CC
S1138700081A20650C352A0000212000FFF7E8FE36
S113871004E0AA68F97A2068FCF780FE00280BD1EF
S1138720019928310978012903D102215434217097
S1138730FEBD54342670FEBD0321009A1170009AC8
S11387409172FEBD80B5010058310A00183212231F
S113875013600123937451600021117496E00000AA
S113876070B502005832110040310023002400BFCC
S113877006A52E5D0E55641C242CFAD31100183165
S113878024240C6001248C74403298E0008004029C
S11387902000000046534C2053454D4946534C207D
S11387A04D4153532053544F52414745303030319B
S11387B0F8B5002300210400583406003936327815
S11387C01506727812042A43B5782F021743F578F8
S11387D03D4302001832D77F282F03D171790F024D
S11387E0B1790AE0A82F09D131790F06717909040A
S11387F03943B7793F020F43F179394318340126DD
S1138800A67412684A432260636026742DE0F8B5AA
S11388100023002104005834060039363278150646
S1138820727812042A43B5782F021743F5783D4332
S113883002001832D77F2A2F03D171790F02B17940
S11388400AE0AA2F09D131790F0671790904394355
S1138850B7793F020F43F17939431834A37412688E
S11388604A432260636001222274A560E160FFF73D
S113887049FEF2BD80B500E080B5010058311831E1
S113888000220A6001238B744A600A74FFF73AFEDF
S113889002BD000070B5020058321100643100239B
S11388A0002400BF9EA52E5D0E55641C082CFAD32F
S11388B01100183108240C6001248C7464324A605D
S11388C00B74FFF71FFE70BD70B505002C00583403
S11388D0200064300021002291A39E5C8654521C27
S11388E0082AFAD320001830082202600122827478
S11388F022006432426001742800FFF703FE383519
S11389002978C90704D5A41C052222702422A27246
S113891070BD10B50021030058331A0018323724F3
S1138920045D252C03D1082414602C3302E00C24AC
S1138930146034335360012393741174FFF7E2FD20
S113894010BD0000F1B588B074A00068029000204A
S1138950002100250022089B5833089C3F342478CA
S11389600194089C143400946C241C5D002C06D0E3
S1138970009CA468002C01D0022400E00324009E83
S113898036680396009E76680496E60002AFFE7091
S1138990009E36680596009E76680696E7000C37BA
S11389A0019EBE4200D93E00009602AEEDB2765D55
S11389B05F186D373E706D1C491C0429F5D30025E2
S11389C005AE765DC9B25F186D373E706D1C491CEB
S11389D0082DF5D36C255D5D002D10D000250BE02E
S11389E003AED2B2B65C5F186D373E70521C491CA0
S11389F0C9B20829F4D36D1CEDB2A542F8DB190005
S1138A001831009A0A6001228A746D334B6008742D
S1138A100898FFF777FD09B0F0BDF8B5040027000A
S1138A2058373800183000250560012686744560E3
S1138A3005742000FFF766FD3834217F02290CD02D
S1138A402178C906C90E172901D12577F2BD2677E9
S1138A50BF1C052139702421B972F2BDF8B5040098
S1138A60270058373B20255C38001830002101606E
S1138A7001268674416001742000FFF743FD6946B6
S1138A80087020003B30407E022809D0354207D0D0
S1138A9020003B304676BF1C052038702420B87275
S1138AA060680368180003D000220721200098475B
S1138AB068460078F2BD80B5DFE670B582B0040088
S1138AC0583026003B3631788907890F6A46117081
S1138AD01830002101600122827441600174200079
S1138AE0FFF710FD0500707E022807D06068036858
S1138AF0180003D06A46082120009847280076BD54
S1138B000100583150300022026001230371052016
S1138B108870202008734A7300207047000000000A
S1138B20000000000000000010B500200022974B58
S1138B30197B974C1B191C78002C00D00122AB4CDC
S1138B4021706270DB7F002B01D01000084310BD40
S1138B50F8B51500002200248C4B1E000836A44FE3
S1138B60DF19012914D0072914D0082921D0092993
S1138B7044D00A2948D00B294CD00C2950D00D29B7
S1138B8054D00E2958D0112922D0122925D059E0C9
S1138B903A7057E0002D55D001203870287878704D
S1138BA029783068FCF74DF92978B06CFDF78EFF11
S1138BB048E03878002845D02A88110A022941DA89
S1138BC05818AE4BC254D2B23068FCF74EF939E0B3
S1138BD0002D37D07878287034E0002D32D02A88E0
S1138BE0110A022908DAFF20000210405918A34A8A
S1138BF0895C0843288025E0052423E0002D21D04A
S1138C002900FEF78CFF1CE0002D1BD02900FEF785
S1138C108CFF16E0002D15D02900FEF791FF10E01F
S1138C20002D0FD02900FEF76BFF0AE0002D09D0BC
S1138C302900FEF767FF04E0002D03D02900FEF7AA
S1138C406CFF04002000F2BD70B582B0684600BF1E
S1138C503FA10A7802704D4E9021C9003000F9F707
S1138C6089FE874CF8F7E2F90028A0680DD1006965
S1138C707821415CEF220A4078300270A0680069D4
S1138C80C16810229143C16030E004697C342188BA
S1138C90A1486288824201D1814209D09F48017271
S1138CA02188090A4172618881726188090AC17246
S1138CB06068AB4D0021C943884205D01021F9F703
S1138CC0E6F9002800D16568A64805608F20C00039
S1138CD0301800210180B16031653160A24C32004E
S1138CE021000020FCF70EFD002801D0012076BDF4
S1138CF02068006930653000FDF7EAFE20684068AE
S1138D00B0603000FCF7C2F86846017849B2FF222F
S1138D108807C00E8240D0430A0004D59349120745
S1138D20120F083A00E092499208920089180A68E2
S1138D3010400860012069460978C906C90E8840B8
S1138D408C4908603068FCF749FB002076BD0000C0
S1138D50180010B50020FCF73DFD002814D10B4C81
S1138D602000FDF7CFFE2000FCF794F8824801684C
S1138D70490309D580214904804A1160804A116061
S1138D800168804A0A40026010BD00006CB2FF1FF7
S1138D905A040000F8B50024144D2C7001266E709E
S1138DA0F9F729FAFDF7B4FE774FB878032802D112
S1138DB0BC70FAF7C9FBF9F724FA3878002800D018
S1138DC0012068702E70F1BD10B5704C0021200098
S1138DD01430F9F7F5F9002120001830F9F7F0F90B
S1138DE014342000F9F7F8F9002010BDECB6FF1F89
S1138DF079040000F7B5002901D0002A01D104202C
S1138E00FEBD002010600127002B02D0012B02D0F0
S1138E102BE0012500E002255D48007800282BD0D6
S1138E205A4C26000836B079002806D024232200A4
S1138E30203202213068FCF7DDF9B7710021C94303
S1138E4020001430F9F7BEF9307EA84205D0012D78
S1138E500BD1022809D14F48FEBDB17EF07E00023D
S1138E6008437169091F814201D20120FEBD2434E7
S1138E7001990C60029908600020FEBD7B0400008B
S1138E8010A0FF1FF7B542480078002841D0212ADE
S1138E9001D30420FEBD002B02D0012B0FD010E023
S1138EA00325F9F7A8F9394C270008370026787903
S1138EB0002808D07E71F9F7A4F93648FEBD0425D0
S1138EC0EFE70120FEBDF9F79CF93D767E76029826
S1138ED0B8760298000AF8760198002808D002981B
S1138EE0002805D00246019920002430F8F7B4FF89
S1138EF04620205C01280CD12423220020320121A9
S1138F003868FCF764F90021C94318342000F9F7E4
S1138F1059F90020FEBD0000FFFF000004A2FF1F5E
S1138F2010B50023002200214469A468A04710BDA5
S1138F30002070472020704710B5144C1648205C60
S1138F40022801D0032807D120001430F9F748F98A
S1138F5020001830F9F744F92068FDF7A3F810BD94
S1138F605CA3FF1F68B2FF1F90A0FF1F1CED00E071
S1138F7000E400E000E100E03480044080E100E02F
S1138F8080E200E0FFFFFBFFC6B6FF1F6CB2FF1FCD
S1138F90ECB6FF1F122700005C04000000F00BF881
S1138FA0002801D000F00AF80020C046C046FAF7B5
S1138FB062FCFAF781FC01207047000010B50749F4
S1138FC079441831064C7C44163404E0081D0A68C0
S1138FD0891888470100A142F8D110BD2804000077
S1138FE03C0400001D22000029220000EC040000C3
S1138FF048A9FF1F68060000CCA0FF1F780A0000E4
S113900000A0FF1F7C050000000A0000D40500003A
S1139010000000000000000000000000000000004C
S1139020000000000000000000000000000000003C
S1139030000000000000000000000000000000002C
S1139040000000000000000000400240000000009A
S113905080A9FF1FC0A9FF1F95010000894D0000D2
S11390600000000084A1FF1F556A000000000000FA
S1139070B0A1FF1F78A0FF1F518B00000200000069
S11390800000000000000000000000002147000074
S11390904147000000000000000000000000000044
S11390A0000000005F670000896700000000000006
S11390B000000000FFFF0100010000002006000086
S11390C000A0FF1FFF1F012001000000E8090000AD
S11390D000000068FFFFFF6F000000008C0A000022
S11390E000000040FFFF074000000000E005000012
S11390F000000840FFEF0F4000000000E005000002
S113910000F00F40FFFF0F4000000000E0050000EA
S1139110000000E0FFFF0FE000000000E005000099
S1139120000000000000000000000000000000003B
S1139130000040018103400002034000830240001C
S113914004024000000000000200000050A1FF1FC4
S1139150000000000300000060A1FF1F01000000E8
S11391600100000070A1FF1F7CA1FF1F010100008E
S1139170000000000200000058A1FF1F00000000D2
S1139180080650018CA1FF1F01000000010000002F
S11391909CA1FF1FA8A1FF1F030100000600FF09F7
S11391A001A101850119012901150026FF00750897
S11391B095239102850219012901150026FF0075E6
S11391C00895239102850319012901150026FF0042
S11391D0750895238102850419012901150026FFCC
S11391E000750895238102C01201000200000040AE
S11391F0A2157300020001020301000009024000ED
S1139200020100C032090400000203000003092126
S113921000010001224C00070581034000010705FD
S11392200203400001090401000208065003070577
S113923083024000000705040240000004030904FF
S11392403A034600520045004500530043004100E4
S11392504C0045002000530045004D0049004300E8
S11392604F004E0044005500430054004F0052008C
S1139270200049004E0043002E0000002A03550040
S113928053004200200043004F004D0050004F00A7
S11392905300490054004500200044004500560096
S11392A049004300450000003E034D0043005500C3
S11392B020004D0053004300200041004E004400B4
S11392C020004800490044002000470045004E00AB
S11392D04500520049004300200044004500560068
S11392E049004300450000002203420041004400BD
S11392F0200053005400520049004E004700000073
S11393000000000000000000000000000400000055
S11393103A0000002A0000003E0000002200000085
S113932058A2FF1F5CA2FF1F98A2FF1FC4A2FF1F29
S113933004A3FF1F3CA3FF1F28A3FF1F0904000071
S113934058A2FF1F0400000050A3FF1F01000000EB
S113935030B504E014780470401C521C491E0029E6
S113936019D0C507F6D40129F4D0850701D40429FE
S113937004D214880480801C921C891E8B08EED0B1
S11393809B00C41803E015680560001D121DA0426F
S1139390F9D3C91AE3E730BD80B513000200180001
S11393A000E080B5FFF7D4FF002002BD10B50C002B
S11393B0110001232200F7F75BF810BDC046C04638
S11393C0C046C046FFF7EAFD70B40121002313E054
S11393D00468001D0C4202D04D466D1E64192360C2
S11393E0241D121F042AFAD22500960701D52380D2
S11393F0AD1C0A4000D02B700268001D002AE7D182
S113940070BC7047C5FFFFFF2005000000A4FF1FCC
S10F9410D00D000020A9FF1F0000000088
S9030411E7
